:020000040800F2
:10000000000008240D2A0008AD250008AF250008CF
:10001000B1250008B3250008B52500080000000040
:10002000000000000000000000000000B7250008EC
:10003000B925000800000000BB250008BD25000808
:100040005D2A00085D2A00085D2A00085D2A000874
:100050005D2A00085D2A0008C52500085D2A000801
:100060005D2A00085D2A00085D2A0008D1250008E5
:100070005D2A00085D2A00085D2A00085D2A000844
:100080005D2A00085D2A00085D2A00085D2A000834
:100090005D2A00085D2A00085D2A00085D2A000824
:1000A0005D2A00085D2A00085D2A00085D2A000814
:1000B0005D2A00085D2A00085D2A00085D2A000804
:1000C0005D2A00085D2A00085D2A00085D2A0008F4
:1000D0005D2A0008E12500085D2A00085D2A000865
:1000E0005D2A00085D2A0008000000005D2A000863
:1000F0005D2A00085D2A00085D2A00085D2A0008C4
:100100005D2A00085D2A00085D2A00085D2A0008B3
:100110005D2A00085D2A00085D2A00085D2A0008A3
:100120005D2A00085D2A00085D2A00085D2A000893
:100130005D2A00085D2A00085D2A00085D2A000883
:1001400000000000000000000000000000000000AF
:100150005D2A00085D2A00085D2A00085D2A000863
:100160005D2A00085D2A00085D2A00085D2A000853
:100170005D2A00085D2A00085D2A00085D2A000843
:100180005D2A00085D2A00085D2A00085D2A000833
:100190005D2A00085D2A00085D2A00085D2A000823
:1001A0005D2A00085D2A00085D2A00085D2A000813
:1001B0005D2A00085D2A00085D2A00085D2A000803
:1001C0005D2A00085D2A00085D2A00085D2A0008F3
:1001D0005D2A00085D2A00085D2A00085D2A0008E3
:1001E0005D2A00085D2A00085D2A00085D2A0008D3
:1001F0005D2A00085D2A00085D2A00085D2A0008C3
:100200005D2A00085D2A00085D2A00085D2A0008B2
:100210005D2A00085D2A00085D2A00085D2A0008A2
:100220005D2A00085D2A00085D2A00080000000021
:100230005D2A00085D2A0008000000005D2A000811
:100240005D2A00085D2A00085D2A00085D2A000872
:100250005D2A00085D2A00085D2A00085D2A000862
:100260005D2A00085D2A00085D2A00085D2A000852
:100270005D2A00085D2A00085D2A000800000000D1
:100280005D2A00085D2A00085D2A000800000000C1
:08029000000000005D2A0008D7
:1002980010B5054C237833B9044B13B10448AFF3B8
:1002A80000800123237010BD6408002400000000B2
:1002B800DC97000808B5034B1BB103490348AFF3AB
:1002C800008008BD0000000068080024DC970008D2
:1002D80081F0004102E000BF83F0004330B54FEAEF
:1002E80041044FEA430594EA050F08BF90EA020F5C
:1002F8001FBF54EA000C55EA020C7FEA645C7FEAEF
:10030800655C00F0E2804FEA5454D4EB5555B8BF11
:100318006D420CDD2C4480EA020281EA030382EA82
:10032800000083EA010180EA020281EA0303362D14
:1003380088BF30BD11F0004F4FEA01314FF4801CE7
:100348004CEA113102D0404261EB410113F0004FF9
:100358004FEA03334CEA133302D0524263EB4303B0
:1003680094EA050F00F0A780A4F10104D5F1200E4E
:100378000DDB02FA0EFC22FA05F2801841F10001A9
:1003880003FA0EF2801843FA05F359410EE0A5F17D
:1003980020050EF1200E012A03FA0EFC28BF4CF0AE
:1003A800020C43FA05F3C01851EBE37101F0004564
:1003B80007D54FF0000EDCF1000C7EEB00006EEB71
:1003C8000101B1F5801F1BD3B1F5001F0CD34908FB
:1003D8005FEA30004FEA3C0C04F101044FEA445252
:1003E80012F5800F80F09A80BCF1004F08BF5FEAD9
:1003F800500C50F1000041EB045141EA050130BDB9
:100408005FEA4C0C404141EB0101013C28BFB1F5CA
:10041800801FE9D291F0000F04BF01460020B1FA15
:1004280081F308BF2033A3F10B03B3F120020CDAE8
:100438000C3208DD02F1140CC2F10C0201FA0CF0C6
:1004480021FA02F10CE002F11402D8BFC2F1200C2B
:1004580001FA02F120FA0CFCDCBF41EA0C019040E1
:10046800E41AA2BF01EB0451294330BD6FEA04042A
:100478001F3C1CDA0C340EDC04F11404C4F1200215
:1004880020FA04F001FA02F340EA030021FA04F327
:1004980045EA030130BDC4F10C04C4F1200220FA7E
:1004A80002F001FA04F340EA0300294630BD21FABC
:1004B80004F0294630BD94F0000F83F4801306BF82
:1004C80081F480110134013D4EE77FEA645C18BF76
:1004D8007FEA655C29D094EA050F08BF90EA020F0D
:1004E80005D054EA000C04BF1946104630BD91EA05
:1004F800030F1EBF0021002030BD5FEA545C05D108
:100508004000494128BF41F0004130BD14F5800446
:100518003CBF01F5801130BD01F0004545F0FE41BA
:1005280041F470014FF0000030BD7FEA645C1ABFEF
:10053800194610467FEA655C1CBF0B46024650EA26
:10054800013406BF52EA033591EA030F41F4002152
:1005580030BD00BF90F0000F04BF0021704730B5D8
:100568004FF4806404F132044FF000054FF00001AD
:1005780050E700BF90F0000F04BF0021704730B56E
:100588004FF4806404F1320410F0004548BF404243
:100598004FF000013EE700BF42004FEAE2014FEA98
:1005A80031014FEA02701FBF12F07F4393F07F4F73
:1005B80081F06051704732F07F4208BF704793F076
:1005C8007F4F04BF41F40021704730B54FF4607489
:1005D80001F0004521F000411CE700BF50EA01028C
:1005E80008BF704730B54FF000050AE050EA010235
:1005F80008BF704730B511F0004502D5404261EBA5
:1006080041014FF4806404F132045FEA915C3FF4E5
:10061800D8AE4FF003025FEADC0C18BF03325FEA82
:10062800DC0C18BF033202EBDC02C2F1200300FA33
:1006380003FC20FA02F001FA03FE40EA0E0021FA58
:1006480002F11444BDE600BF70B54FF0FF0C4CF446
:10065800E06C1CEA11541DBF1CEA135594EA0C0FF8
:1006680095EA0C0F00F0DEF82C4481EA030621EA33
:100678004C5123EA4C5350EA013518BF52EA03356E
:1006880041F4801143F4801338D0A0FB02CE4FF020
:100698000005E1FB02E506F00042E0FB03E54FF050
:1006A8000006E1FB03569CF0000F18BF4EF0010E48
:1006B800A4F1FF04B6F5007F64F5407404D25FEA44
:1006C8004E0E6D4146EB060642EAC62141EA5551F7
:1006D8004FEAC52040EA5E504FEACE2EB4F1FD0C39
:1006E80088BFBCF5E06F1ED8BEF1004F08BF5FEAB7
:1006F800500E50F1000041EB045170BD06F0004669
:1007080046EA010140EA020081EA0301B4EB5C0415
:10071800C2BFD4EB0C0541EA045170BD41F480110D
:100728004FF0000E013C00F3AB8014F1360FDEBF32
:10073800002001F0004170BDC4F10004203C35DA0E
:100748000C341BDC04F11404C4F1200500FA05F391
:1007580020FA04F001FA05F240EA020001F0004232
:1007680021F0004110EBD37021FA04F642EB0601A8
:100778005EEA430E08BF20EAD37070BDC4F10C04D2
:10078800C4F1200500FA04F320FA05F001FA04F296
:1007980040EA020001F0004110EBD37041F1000182
:1007A8005EEA430E08BF20EAD37070BDC4F120058D
:1007B80000FA05F24EEA020E20FA04F301FA05F2F5
:1007C80043EA020321FA04F001F0004121FA04F29D
:1007D80020EA020000EBD3705EEA430E08BF20EA6D
:1007E800D37070BD94F0000F0FD101F000464000A7
:1007F80041EB010111F4801F08BF013CF7D041EA29
:10080800060195F0000F18BF704703F0004652002C
:1008180043EB030313F4801F08BF013DF7D043EAFD
:100828000603704794EA0C0F0CEA135518BF95EAB3
:100838000C0F0CD050EA410618BF52EA4306D1D13A
:1008480081EA030101F000414FF0000070BD50EA59
:10085800410606BF1046194652EA430619D094EAE3
:100868000C0F02D150EA013613D195EA0C0F05D1CD
:1008780052EA03361CBF104619460AD181EA030121
:1008880001F0004141F0FE4141F470014FF00000D9
:1008980070BD41F0FE4141F4780170BD70B54FF074
:1008A800FF0C4CF4E06C1CEA11541DBF1CEA1355F4
:1008B80094EA0C0F95EA0C0F00F0A7F8A4EB0504D6
:1008C80081EA030E52EA03354FEA013100F08880CD
:1008D8004FEA03334FF0805545EA131343EA126396
:1008E8004FEA022245EA111545EA10654FEA00264B
:1008F8000EF000419D4208BF964244F1FD0404F504
:10090800407402D25B084FEA3202B61A65EB03055F
:100918005B084FEA32024FF480104FF4002CB6EB1C
:10092800020E75EB030E22BFB61A754640EA0C009C
:100938005B084FEA3202B6EB020E75EB030E22BFDC
:10094800B61A754640EA5C005B084FEA3202B6EB1D
:10095800020E75EB030E22BFB61A754640EA9C00DC
:100968005B084FEA3202B6EB020E75EB030E22BFAC
:10097800B61A754640EADC0055EA060E18D04FEA6A
:10098800051545EA16754FEA06164FEAC30343EA0A
:1009980052734FEAC2025FEA1C1CC0D111F4801FD7
:1009A8000BD141EA00014FF000004FF0004CB6E7D0
:1009B80011F4801F04BF01430020B4F1FD0C88BF6F
:1009C800BCF5E06F3FF6AFAEB5EB030C04BFB6EB7A
:1009D800020C5FEA500C50F1000041EB045170BD6D
:1009E8000EF0004E4EEA113114EB5C04C2BFD4EB9A
:1009F8000C0541EA045170BD41F480114FF0000E1E
:100A0800013C90E645EA060E8DE60CEA135594EA99
:100A18000C0F08BF95EA0C0F3FF43BAF94EA0C0F9C
:100A28000AD150EA01347FF434AF95EA0C0F7FF411
:100A380025AF104619462CE795EA0C0F06D152EA65
:100A480003353FF4FDAE1046194622E750EA410649
:100A580018BF52EA43067FF4C5AE50EA41047FF45A
:100A68000DAF52EA43057FF4EBAE12E74FF0FF3CBF
:100A780006E000BF4FF0010C02E000BF4FF0010C90
:100A88004DF804CD4FEA410C7FEA6C5C4FEA430C09
:100A980018BF7FEA6C5C1BD001B050EA410C0CBF58
:100AA80052EA430C91EA030F02BF90EA020F0020BA
:100AB800704710F1000F91EA030F58BF994208BF21
:100AC80090422CBFD8176FEAE37040F001007047DE
:100AD8004FEA410C7FEA6C5C02D150EA013C07D135
:100AE8004FEA430C7FEA6C5CD6D152EA033CD3D080
:100AF8005DF8040B704700BF8446104662468C467A
:100B08001946634600E000BF01B5FFF7B7FF0028AC
:100B180048BF10F1000F01BD4DF808EDFFF7F4FFD5
:100B28000CBF012000205DF808FB00BF4DF808ED60
:100B3800FFF7EAFF34BF012000205DF808FB00BF83
:100B48004DF808EDFFF7E0FF94BF012000205DF8A5
:100B580008FB00BF4DF808EDFFF7CEFF94BF01205A
:100B680000205DF808FB00BF4DF808EDFFF7C4FF53
:100B780034BF012000205DF808FB00BF4FEA4102A6
:100B880012F5001215D211D56FF47873B3EB6252D7
:100B980012D94FEAC12343F0004343EA505311F0FE
:100BA800004F23FA02F018BF404270474FF0000090
:100BB800704750EA013005D111F0004008BF6FF0CE
:100BC800004070474FF00000704700BF4A0011D244
:100BD80012F5001211D20DD56FF47873B3EB62528F
:100BE8000ED44FEAC12343F0004343EA505323FA9B
:100BF80002F070474FF00000704750EA013002D110
:100C08004FF0FF3070474FF0000070474FEA410245
:100C1800B2F1E04324BFB3F5001CDCF1FE5C0DD952
:100C280001F0004C4FEAC0024CEA5070B2F1004F9C
:100C380040EB830008BF20F00100704711F0804F9F
:100C480021D113F13872BCBF01F00040704741F464
:100C580080114FEA5252C2F11802C2F1200C10FA68
:100C68000CF320FA02F018BF40F001004FEAC1234C
:100C78004FEAD32303FA0CFC40EA0C0023FA02F3F0
:100C88004FEA4303CCE77FEA625307D150EA0133C6
:100C98001EBF4FF0FE4040F44000704701F0004096
:100CA80040F0FE4040F40000704700BF80F0004074
:100CB80002E000BF81F0004142001FBF5FEA41032C
:100CC80092EA030F7FEA226C7FEA236C6AD04FEA2C
:100CD8001262D2EB1363C1BFD21841404840414071
:100CE800B8BF5B42192B88BF704710F0004F40F423
:100CF800000020F07F4018BF404211F0004F41F43F
:100D0800000121F07F4118BF494292EA030F3FD00A
:100D1800A2F1010241FA03FC10EB0C00C3F120031D
:100D280001FA03F100F0004302D5494260EB4000AC
:100D3800B0F5000F13D3B0F1807F06D340084FEA17
:100D4800310102F10102FE2A51D2B1F1004F40EB0C
:100D5800C25008BF20F0010040EA03007047490074
:100D680040EB0000013A28BFB0F5000FEDD2B0FA11
:100D780080FCACF1080CB2EB0C0200FA0CF0AABF34
:100D880000EBC25052421843BCBFD04018437047D2
:100D980092F0000F81F4000106BF80F400000132D8
:100DA800013BB5E74FEA41037FEA226C18BF7FEAAF
:100DB800236C21D092EA030F04D092F0000F08BFF1
:100DC8000846704790EA010F1CBF0020704712F0D8
:100DD8007F4F04D1400028BF40F00040704712F117
:100DE80000723CBF00F50000704700F0004343F07C
:100DF800FE4040F4000070477FEA226216BF0846B2
:100E08007FEA23630146420206BF5FEA412390EA74
:100E1800010F40F4800070474FF0000304E000BF6A
:100E280010F0004348BF40425FEA000C08BF70471B
:100E380043F0964301464FF000001CE050EA0102DF
:100E480008BF70474FF000030AE000BF50EA0102F4
:100E580008BF704711F0004302D5404261EB4101E1
:100E68005FEA010C02BF84460146002043F0B64306
:100E780008BFA3F18053A3F50003BCFA8CF2083A2B
:100E8800A3EBC25310DB01FA02FC634400FA02FC34
:100E9800C2F12002BCF1004F20FA02F243EB02003B
:100EA80008BF20F00100704702F1200201FA02FC9D
:100EB800C2F1200250EA4C0021FA02F243EB020090
:100EC80008BF20EADC7070474FF0FF0C1CEAD052D4
:100ED8001EBF1CEAD15392EA0C0F93EA0C0F6FD095
:100EE8001A4480EA010C400218BF5FEA41211ED073
:100EF8004FF0006343EA501043EA5111A0FB01315F
:100F08000CF00040B1F5000F3EBF490041EAD37133
:100F18005B0040EA010062F17F02FD2A1DD8B3F1AF
:100F2800004F40EBC25008BF20F00100704790F01E
:100F3800000F0CF0004C08BF49024CEA502040EA70
:100F480051207F3AC2BFD2F1FF0340EAC250704736
:100F580040F400004FF00003013A5DDC12F1190F74
:100F6800DCBF00F000407047C2F10002410021FAE6
:100F780002F1C2F1200200FA02FC5FEA310040F1FE
:100F8800000053EA4C0308BF20EADC70704792F077
:100F9800000F00F0004C02BF400010F4000F013AAF
:100FA800F9D040EA0C0093F0000F01F0004C02BFAA
:100FB800490011F4000F013BF9D041EA0C018FE719
:100FC8000CEAD15392EA0C0F18BF93EA0C0F0AD01F
:100FD80030F0004C18BF31F0004CD8D180EA010045
:100FE80000F00040704790F0000F17BF90F0004FDE
:100FF800084691F0000F91F0004F14D092EA0C0FC0
:1010080001D142020FD193EA0C0F03D14B0218BF52
:10101800084608D180EA010000F0004040F0FE4098
:1010280040F40000704740F0FE4040F44000704734
:101038004FF0FF0C1CEAD0521EBF1CEAD15392EAB3
:101048000C0F93EA0C0F69D0A2EB030280EA010CA3
:1010580049024FEA402037D04FF0805343EA11113C
:1010680043EA10130CF000408B4238BF5B0042F19A
:101078007D024FF4000C8B4224BF5B1A40EA0C003F
:10108800B3EB510F24BFA3EB510340EA5C00B3EB71
:10109800910F24BFA3EB910340EA9C00B3EBD10F5F
:1010A80024BFA3EBD10340EADC001B0118BF5FEAB1
:1010B8001C1CE0D1FD2A3FF650AF8B4240EBC250DA
:1010C80008BF20F0010070470CF0004C4CEA50209B
:1010D8007F32C2BFD2F1FF0340EAC250704740F4EA
:1010E80000004FF00003013A37E792F0000F00F0DC
:1010F800004C02BF400010F4000F013AF9D040EA5A
:101108000C0093F0000F01F0004C02BF490011F4ED
:10111800000F013BF9D041EA0C0195E70CEAD153E5
:1011280092EA0C0F08D142027FF47DAF93EA0C0FCC
:101138007FF470AF084676E793EA0C0F04D14B02B0
:101148003FF44CAF08466EE730F0004C18BF31F062
:10115800004CCAD130F000427FF45CAF31F000435C
:101168007FF43CAF5FE700BF42000ED2B2F1FE4F02
:101178000BD34FF09E03B3EB126209D44FEA00235E
:1011880043F0004323FA02F070474FF00000704725
:1011980012F1610F01D1420202D14FF0FF307047C6
:1011A8004FF00000704700BF53B94AB9002908BF83
:1011B80000281CBF4FF0FF314FF0FF3000F074B92A
:1011C800ADF1080C6DE904CE00F006F8DDF804E096
:1011D800DDE9022304B070472DE9F047089E0D466B
:1011E80004468846002B4DD18A42944668D9B2FA03
:1011F80082F252B101FA02F3C2F1200120FA01F1A0
:101208000CFA02FC41EA030894404FEA1C45210C01
:10121800B8FBF5FE1FFA8CF705FB1E8341EA034372
:101228000EFB07F199420BD91CEB03030EF1FF30BB
:1012380080F01E81994240F21B81AEF1020E634498
:101248005B1AA4B2B3FBF5F005FB103344EA034480
:1012580000FB07F7A7420AD91CEB040400F1FF338F
:1012680080F00881A74240F2058164440238E41BFB
:1012780040EA0E4000211EB1D4400023C6E90043D5
:10128800BDE8F0878B4208D9002E00F0EE800021DF
:10129800C6E900050846BDE8F087B3FA83F10029DE
:1012A8004AD1AB4202D3824200F2F980841A65EB3C
:1012B800030301209846002EE2D0C6E90048DFE784
:1012C80002B9FFDEB2FA82F2002A40F09180A1EB67
:1012D8000C054FEA1C471FFA8CFE0121B5FBF7F3FA
:1012E80007FB1350250C45EA00450EFB03F0A84206
:1012F80008D91CEB050503F1FF3802D2A84200F219
:10130800CB8043462D1AA4B2B5FBF7F007FB105566
:1013180044EA05440EFB00FEA64508D91CEB04046C
:1013280000F1FF3502D2A64500F2BB802846A4EBA7
:101338000E0440EA03409EE7C1F120078B4022FAE1
:1013480007FC4CEA030C20FA07F405FA01F31C43E6
:10135800FD404FEA1C4900FA01F3B5FBF9F8200CEF
:101368001FFA8CFE09FB185540EA054508FB0EF0EC
:10137800A84202FA01F20BD91CEB050508F1FF3A65
:1013880080F08880A84240F28580A8F10208654470
:101398002D1AA4B2B5FBF9F009FB105544EA05452E
:1013A80000FB0EFEAE4508D91CEB050500F1FF3425
:1013B8006CD2AE456AD90238654440EA0840A0FBC1
:1013C8000294A5EB0E05A542C846A64656D353D0AF
:1013D8005EB1B3EB080265EB0E0505FA07F722FAD2
:1013E80001F3CD401F43C6E900750021BDE8F08731
:1013F800C2F1200320FA03F10CFA02FC25FA03F3E8
:1014080095400D434FEA1C471FFA8CFEB3FBF7F1DA
:1014180007FB11302B0C43EA004301FB0EF0984206
:1014280004FA02F408D91CEB030301F1FF382FD2A8
:1014380098422DD9023963441B1AADB2B3FBF7F0B9
:1014480007FB103345EA034500FB0EF3AB4208D90E
:101458001CEB050500F1FF3816D2AB4214D902384F
:101468006544ED1A40EA014138E73146304607E75E
:101478008646E5E61846FAE64B45A9D2B9EB0208D6
:1014880064EB0C0E0138A3E74046EAE7204694E7F0
:101498004146D1E7D0467BE7023B654432E7084640
:1014A80009E76444023842E7704700BF844641EACE
:1014B800000313F003036DD1403A41D351F8043BC4
:1014C80040F8043B51F8043B40F8043B51F8043B16
:1014D80040F8043B51F8043B40F8043B51F8043B06
:1014E80040F8043B51F8043B40F8043B51F8043BF6
:1014F80040F8043B51F8043B40F8043B51F8043BE6
:1015080040F8043B51F8043B40F8043B51F8043BD5
:1015180040F8043B51F8043B40F8043B51F8043BC5
:1015280040F8043B51F8043B40F8043B51F8043BB5
:1015380040F8043B51F8043B40F8043B403ABDD224
:10154800303211D351F8043B40F8043B51F8043BC6
:1015580040F8043B51F8043B40F8043B51F8043B85
:1015680040F8043B103AEDD20C3205D351F8043B55
:1015780040F8043B043AF9D2043208D0D2071CBF21
:1015880011F8013B00F8013B01D30B88038060464A
:10159800704700BF082A13D38B078DD010F00303C0
:1015A8008AD0C3F10403D21ADB071CBF11F8013B30
:1015B80000F8013B80D331F8023B20F8023B7BE77F
:1015C800043AD9D3013A11F8013B00F8013BF9D2AA
:1015D8000B7803704B7843708B7883706046704744
:1015E80000B587B0002301930293039304930593F6
:1015F800022301930123029301A9034802F0AAFFE1
:1016080007B05DF804FB00BF0008025800B587B0BA
:1016180000230193029303930493059302230193F8
:1016280001A9034802F096FF07B05DF804FB00BF6C
:101638000008025810B5FFF7D3FF094C0022022119
:10164800204603F0A2F840F2EE2000F029FB012228
:101658000221204603F099F80F2000F021FB10BD6D
:101668000008025810B5FFF7D1FF002402211248E4
:1016780003F084F838B1C72C05D80134E4B201204E
:1016880000F00EFBF2E7C72C13D8002404E0013465
:10169800E4B2012000F004FB0221074803F06EF8D1
:1016A80008B9EF2CF3D94FF4F07000F0F9FA0120E3
:1016B80010BD0020FCE700BF0008025810B5FFF776
:1016C8008FFF0F4C00220221204603F05EF8022013
:1016D80000F0E6FA01220221204603F056F8FFF74F
:1016E80095FF0C2000F0DCFA0221204603F046F8B2
:1016F800044600B10124322000F0D2FA204610BD81
:101708000008025838B500252C4607E0FFF7D6FF39
:10171800640844EAC014E4B20135EDB2072DF5D9E6
:10172800204638BD70B50546FFF75AFF002413E080
:10173800154E00220221304603F027F83C2000F025
:10174800AFFA01220221304603F01FF8022000F010
:10175800A7FA6D080134E4B2072C14D815F0010F6C
:10176800E6D0094E00220221304603F00EF802208E
:1017780000F096FA01220221304603F006F83C20D8
:1017880000F08EFAE5E770BD0008025808B5FFF7CB
:1017980051FFFFF767FFCC20FFF7C4FF4420FFF796
:1017A800C1FF08BD70B586B000F072FA002301933E
:1017B8000293039304930593124BD3F8E02042F06D
:1017C8000402C3F8E020D3F8E03003F004030093E8
:1017D800009B02250195012602960B4C01A9204683
:1017E80002F0B8FE32462946204602F0CEFF4FF4FA
:1017F8007A7001F099F9FFF71DFFFFF733FF06B084
:1018080070BD00BF004402580008025808B5FFF731
:10181800E7FE01220221024802F0B7FF08BD00BF1F
:101828000008025838B5FFF7B1FFFFF703FFFFF7CD
:1018380019FFCC20FFF776FFBE20FFF773FFFFF7F5
:1018480061FF0546FFF75EFF0446FFF7DFFFA4B21E
:101858002402A4B214FA85F4A0B204F47844B4F5CE
:10186800784F08D0FEF786FE0022084BFEF7ECFE04
:10187800FFF7CCF938BD404280B2FEF77BFE00226C
:10188800034BFEF7E1FEFFF7C1F9F3E70000B03FB5
:101898000000B0BF00B586464FF0000C604611E06E
:1018A8000133DBB2072B09D800F001024008002AF7
:1018B800F6D048F20842424090B2F1E70CF1010C30
:1018C8001FFA8CFC8C4504D21EF80C3058400023BB
:1018D800E8E75DF804FB1BB338B50C4611461D4616
:1018E800231E18BF0123002A18BF0023DBB9552384
:1018F8002B70AA236B70A870230AEB702C7154B953
:101908002146681DFFF7C6FF631D020AEA54A31D9E
:10191800E854E01D38BD2246681DFFF7C7FDEFE714
:101928004FF0FF3070474FF0FF30F3E72DE9F843F1
:10193800002B18BF002831D0174606469846037872
:10194800552B2ED14378AA2B2ED10479C37804EBDA
:101958000324A4B20639A146A14228DD03199D79C2
:10196800EE2D0FD02146701DFFF794FF33195B79D8
:1019780005EB0325A8421DD144B94FF0000948469C
:10198800BDE8F8835B79EE2BECD1F5E7B3783B70D3
:101998002246711D4046FFF789FDF0E7DFF81C90ED
:1019A800EDE7DFF81C90EAE7DFF81490E7E76FF05F
:1019B800C709E4E7DFF80C90E1E700BF0CFEFFFF82
:1019C800D4FEFFFFA8FDFFFF08B5012802D00228BA
:1019D80006D008BD01220221044802F0D6FEF8E72D
:1019E80001221146014802F0D0FEF2E7000C02582D
:1019F80008B5012802D0022806D008BD002202211D
:101A0800044802F0C2FEF8E700220121014802F072
:101A1800BCFEF2E7000C025800B583B04FF47A73AD
:101A280003FB00F0C0F307638DF80430C0F30743ED
:101A38008DF80530C0F307238DF806308DF80700C0
:101A480007480268136843F0010313606423042203
:101A58000DEB020106F0B3F803B05DF804FB00BF1C
:101A68008C430024000000002DE9F04D0E46154679
:101A78001F46FEF77FFD26A3D3E90023FEF7E4FD0A
:101A88000022274BFEF70AFFFFF778F880464FF051
:101A9800000C644601E00CF1010CAC4505D236F8A7
:101AA8001CE0A645F7DD7446F5E7632F94BF0023D5
:101AB80001230A2F98BF43F001032BBB2046FEF7F2
:101AC80059FD82468B464046FEF754FD12A3D3E9E2
:101AD8000023FEF7B9FD02460B4650465946FFF76C
:101AE80025F828B9444503DC00242046BDE8F08DDC
:101AF80007FB04F4B4FBF8F42046FFF78DFF4FF41E
:101B08007A7001F011F8F0E70024EEE7AFF30080F7
:101B180000000000E0FFEF40666666666666EE3F1E
:101B2800000059402DE9F04F85B082468B46164695
:101B38001F46894600290BDB4FEA6909C9F10004F1
:101B480000220023CDE90023D046CA46D9462AE020
:101B580001F10109F0E704FB04FBCBF1000B32466D
:101B68003B4630463946FEF7B9FB32463B46FEF760
:101B78006BFDCDE9020104EB0A0508EBC5055846E3
:101B8800FEF7F8FCDDE90223FEF788FE07F0DCFB30
:101B980002460B46C5E90023DDE90001FEF79EFB7E
:101BA800CDE9000101345445D5DDC246CB460024B9
:101BB800DDE900670AE00AEBC40532463B46D5E991
:101BC8000001FEF76BFEC5E9000101345C45F2DB5C
:101BD80005B0BDE8F08F00002DE9F04F8FB0074643
:101BE800039116460022264B052104A8FFF79AFF09
:101BF8004FF0000B5D4634E00134022C23DC2B1936
:101C0800002BA8BF9E42F7DDA21C0EA901EBC20261
:101C180052E90AAB37F81300FEF7ACFC52465B46B4
:101C2800FEF712FD02460B46DDE90001FEF756FB02
:101C3800CDE9000152465B4640464946FEF74EFB59
:101C480080468946D8E742464B46DDE90001FEF763
:101C580025FE07F02FFBFEF7B9FF039B23F81500BD
:101C68000135B54208DA6FF001044FF000084FF073
:101C78000009CDE90089C0E70FB0BDE8F08F00BFCB
:101C88000000F83F08B50222FFF7A6FF08BD0000D4
:101C980008B5024804F0F2FB08BD00BF3842002432
:101CA80038B504460C4A156800226A620AE0686A78
:101CB800FEF750FC06A3D3E90023FEF7C5FCFEF7A8
:101CC80085FF0346A342F2D338BD00BFAFF30080BF
:101CD8009A9999999999B93F3842002408B50848C2
:101CE8000268136823F0010313604FF48162054909
:101CF80006F06CF9044A936843F08003936008BDCA
:101D08008C430024E43C00240044004070B5ADF549
:101D1800006D04460E4615462E4B1A682E4B9A4205
:101D28001CD92E4B1B68C3F3C0634BB12A4B9A4294
:101D380032D92A4B4FF000625A60294804F02EFE2F
:101D48006B46324629462046FFF7C5FD82B26946F2
:101D5800234804F0C7FD0DF5006D70BD214B9A4274
:101D680004D9583B5B68C3F3C063DEE71E4B9A4255
:101D780005D903F552731B68C3F3C063D5E71B4B42
:101D88009A4204D9583B5B68C3F3C063CDE7184B4C
:101D98001B68C3F3C063C8E7124B9A4204D9583B87
:101DA8004FF00062DA60C8E70F4B9A4205D903F595
:101DB80052734FF000629A60BFE70C4B9A4204D905
:101DC800583B4FF00062DA60B7E7094B4FF000620A
:101DD8009A60B2E7BC410024B8040240005402589B
:101DE800FC42002458040240B80002405800024057
:101DF80000000240F8B504460268164B9A4204D027
:101E08002268154B9A4218D0F8BD144D2A681368F9
:101E180023F001031360124E4FF481673A46311DD7
:101E28001048FFF743FB104A1368013313603A4622
:101E38003146284606F0CAF8E2E70C4A13880C49EE
:101E48000C780C48C4540133138001220A4806F068
:101E580035F8D9E700440040001001408C430024C5
:101E6800E43C0024D0380024D83C0024B8410024A5
:101E7800EC400024F0400024FC420024012800D05B
:101E88007047034B1A68136843F001031360F7E7C0
:101E98008C4300247C4B1988072900D8704710B55B
:101EA800B6B0C1F30D0400218DF807100491C422C7
:101EB80005A806F075F904AB0DF107022146734831
:101EC800FFF734FD002855DD9DF80730503B122BF5
:101ED80050D8DFE803F00A59717A8DA5AF4F4F4FFC
:101EE8004F4F4F4F4F4FB9C7CD0049238DF808309A
:101EF80053238DF8093033238DF80A302D238DF8BC
:101F08000B30634B19686348A0FB01308009624BB2
:101F1800A3FB0042D20802EB8202A0EB420230325D
:101F28008DF80C205D48A0FB01204009A3FB00426E
:101F3800D20802EB8202A0EB420230328DF80D206B
:101F4800A3FB0102D208A3FB0203DB0803EB830314
:101F5800A2EB430330338DF80E3002EB8202A1EB83
:101F6800420130318DF80F1008220DEB020150208C
:101F7800FFF7CCFEC8220021444806F011F9424B75
:101F880000221A8036B010BD9DF810309DF811005F
:101F9800000440EA03609DF8123040EA03209DF8EF
:101FA800133018433E4B1860FFF736FD042204A98E
:101FB8005120FFF7ABFEDDE73A4B00221A60012201
:101FC80004A95220FFF7A2FED4E7354B1B688DF811
:101FD8000B301A0A8DF80A201A0C8DF809201B0EEE
:101FE8008DF80830042202A95320FFF78FFEC1E7BD
:101FF800FFF718FC2C4B1860C0F307638DF8083006
:10200800C0F307438DF80930C0F307238DF80A3071
:102018008DF80B00042202A95420FFF777FEA9E7E8
:102028009DF81000FFF7D0FC012204A95520FFF706
:102038006DFE9FE79DF81000FFF7DAFC012204A966
:102048005620FFF763FE95E79DF81020174B1A708E
:102058009DF91420164B1A70052204A96020FFF779
:1020680055FE87E7114A137863F07F03137081E701
:102078000E4B1B7803F07F038DF80830012202A96C
:102088006220FFF743FE75E7B8410024F0400024C2
:102098000C000024D34D6210CDCCCCCC1F85EB5165
:1020A8000800002404000024E03C0024DC3C002458
:1020B8000000002470B5ADF5816D022000F04EFDE2
:1020C80001226949694805F0F9FE694B186800233F
:1020D80002221946806806F0B5F82A21654800F002
:1020E800E5F8FFF75FFBFFF7F9FD0F20FFF794FC1A
:1020F80000252C460AE0604B01221A60C822002104
:102108005E4806F04DF85E4B00221A805A4B1B6859
:10211800002B49D1FFF7BEFE5A4B1A685A4B1B6871
:102128009A42F3D0594B1B684FF4017258495A2010
:10213800FFF79AFC0028DED0544B1860DEE75549BB
:1021480031F81300524A32F8132004FB0022B2FB84
:10215800F6F221F813200133B3F5017FEFD33446AB
:1021680034E00023F8E703EB032203EB42020244C6
:10217800494931F81220494E4949A1FB022136F854
:10218800102002EBD10226F810200133092BEAD9DE
:102198000130B0F5017F01D20023F7E7414A1378F7
:1021A80092F90020002A24DB334B1B68012BADD1A8
:1021B800FFF770FE334B1A68334B1B689A42EDD019
:1021C800661C394B1B78B342CBD20024344BA3FB9B
:1021D8000523DB0803EB8303A5EB43034FF481627C
:1021E8002B492E4800EB4300FFF760F9013500202A
:1021F800CFE703F07F032B4A1370042B0AD8DFE8DC
:1022080003F0030F16212C0040F2064220496120FA
:10221800FFF77CFD234A137803F07F031370C3E7AD
:1022280040F206421B496120FFF770FDF2E769465C
:102238001748FFF727FD40F2064269466120FFF77D
:1022480065FDE7E769461348FFF71CFD40F20642C3
:1022580069466120FFF75AFDDCE740F206420F4964
:102268006120FFF753FDD5E7EC400024FC42002431
:1022780020000024B804024004000024F040002498
:10228800B8410024D83C0024880C0024080000240D
:10229800D038002480080024941000248C0C0024DA
:1022A800CDCCCCCCDC3C00240000002410B582B09E
:1022B8001E4B98422CD91E4BD3F8D82042F002026C
:1022C800C3F8D820D3F8D83003F002030093009B5A
:1022D800184B194C9C67A363206061604023A3607E
:1022E8000023E3604FF4806222616361A361E361CC
:1022F8004FF48032226263620322A262E3622363A4
:10230800204601F07BF8204600F0A6FE02B010BD82
:10231800074BD3F8D82042F00102C3F8D820D3F8ED
:10232800D83003F001030193019BD1E70004024078
:1023380000440258FC420024BC41002400B583B08C
:102348000B4BD3F8D82042F00102C3F8D820D3F8B9
:10235800D83003F001030193019B002211460B20A2
:1023680000F00EFC0B2000F041FC03B05DF804FB0C
:102378000044025870B588B000240394049405946E
:10238800069407942A4BD3F8E02042F08002C3F861
:10239800E020D3F8E02002F080020092009AD3F8FF
:1023A800E02042F00102C3F8E020D3F8E02002F078
:1023B80001020192019AD3F8E02042F00202C3F828
:1023C800E020D3F8E03003F002030293029B194D9A
:1023D80022464FF40071284602F0D7F901260396E9
:1023E8004FF404130493059403A9134802F0B2F8B8
:1023F8004FF48043039302230493059406940793B0
:1024080003A9284602F0A6F84FF400730393049634
:102418000594069403A9284602F09CF82246214612
:10242800062000F0ADFB062000F0E0FB08B070BD10
:1024380000440258000402580000025872B6FEE731
:1024480000B59FB04C2200210BA805F0A9FE202260
:10245800002103A805F0A4FE022002F0ABF9002336
:102468000093394BDA6A22F00102DA62DB6A03F080
:1024780001030093354B9A6942F440429A619B6983
:1024880003F440430093009B304B9B6913F4005FB7
:10249800FAD02F4BD3F8F42042F00202C3F8F4200C
:1024A800D3F8F43003F002030193019B0023029355
:1024B800264B9A6942F440429A619B6903F440436F
:1024C8000293214BDA6A42F00102DA62DB6A03F016
:1024D80001030293029B1D4B9B6913F4005FFAD022
:1024E80001230B934FF480330C9302231493159319
:1024F80005221692C02217921893062219921A934F
:1025080008231B9300231C931D930BA802F07CF94E
:10251800B0B93F23039303230493002305930823AF
:1025280006934023079308934FF4806209920A9315
:10253800042103A802F0AEFD20B91FB05DF804FB2A
:10254800FFF77CFFFFF77AFF0004005800480258A5
:102558000044025808B500F0A7FA4FF4FA6000F0FA
:10256800E3FAFFF76DFFFFF705FF00F02BF9FFF720
:10257800E5FE00F05BF900F0D3F8FFF79BFDFEE7FE
:1025880082B0074BD3F8F42042F00202C3F8F420DB
:10259800D3F8F43003F002030193019B02B07047B3
:1025A80000440258FEE7FEE7FEE7FEE7FEE7704755
:1025B8007047704708B500F0A5FA08BD08B50120B6
:1025C80002F0E9F808BD000008B5024801F024FC53
:1025D80008BD00BF8442002408B5024804F0AAFAE6
:1025E80008BD00BFFC42002470B50C461646002505
:1025F80006E0AFF30080214601F8010B01350C46D7
:10260800B542F6DB304670BD4FF0FF3070474FF4EF
:1026180000534B60002070470020704710B50346F8
:102628000C4A0D490D48006840B10C480068034445
:10263800521A934206D8094A136010BD0748084C3D
:102648000460F2E705F082FD0C2303604FF0FF30D1
:10265800F3E700BF0000082400040000344200240F
:1026680068440024244B1B6803F00F03062B06D88C
:10267800214A136823F00F0343F0070313601F4B2D
:102688001A6842F001021A6000221A6119681C4A8D
:102698000A401A60184B1B6813F0080F06D0164A38
:1026A800136823F00F0343F007031360134B002252
:1026B8009A61DA611A62134999621349D962134916
:1026C80019635A639963DA6319645A64196821F4BF
:1026D800802119601A660E4B1A680E4B1340B3F12D
:1026E800005F03D20C4B0122C3F808210B4B43F2C5
:1026F800D2021A60704700BF0020005200440258FE
:102708007FEDF6EA000202020000FF0180020101EB
:102718000010005C0000FFFF0080005100400052E4
:1027280000B589B00023049305930693079301939A
:10273800029303931448154A02601722426083608B
:102748004FF0FF32C2600361836103F05DFF90B90F
:102758004FF48053049304A90B4803F091FF68B920
:1027680000230193039301A9074804F025F840B911
:1027780009B05DF804FBFFF761FEE9E7FFF75EFECD
:10278800EEE7FFF75BFEF3E738420024000C004059
:1027980002680A4B9A4200D0704782B0084BD3F8BF
:1027A800E82042F00802C3F8E820D3F8E83003F044
:1027B80008030193019B02B0704700BF000C004062
:1027C8000044025808B51748174B03604FF46123BB
:1027D800436000238360C36003610C22426183610C
:1027E800C36103624362836205F090FA70B9002105
:1027F8000C4805F061FC60B900210A4805F081FC2D
:1028080050B9084805F039FC48B908BDFFF716FE6D
:10281800EDE7FFF713FEEFE7FFF710FEF1E7FFF72D
:102828000DFEF2E7FC4200240010014008B51748ED
:10283800174B03604FF46123436000238360C36038
:1028480003610C2242618361C36103624362836254
:1028580005F05CFA70B900210C4805F02DFC60B950
:1028680000210A4805F04DFC50B9084805F005FC60
:1028780048B908BDFFF7E2FDEDE7FFF7DFFDEFE739
:10288800FFF7DCFDF1E7FFF7D9FDF2E78C43002401
:102898000044004030B5B9B004460021339134916A
:1028A800359136913791BC2204A805F079FC23684C
:1028B800444A934204D0444A93423AD039B030BD96
:1028C8000123049304A802F081FE78BB3F4BD3F8A0
:1028D800F02042F01002C3F8F020D3F8F02002F004
:1028E80010020092009AD3F8E02042F00102C3F8E7
:1028F800E020D3F8E03003F001030193019B4FF48B
:10290800C063339302233493002435943694072309
:10291800379333A92E4801F01DFE22462146252073
:1029280000F02EF9252000F061F9C7E7FFF786FDD2
:10293800CCE70223049304A802F048FE00283BD108
:10294800224BD3F8E82042F40032C3F8E820D3F849
:10295800E82002F400320292029AD3F8E02042F012
:102968000102C3F8E020D3F8E03003F00103039339
:10297800039B0C2333930223349300253595369516
:102988000723379333A9124801F0E4FD1148124B8D
:1029980003602B2343608560C5604FF48063036147
:1029A80045618561C5610562456200F055FB30B936
:1029B800084BE3679C6381E7FFF740FDC0E7FFF73B
:1029C8003DFDF5E700100140004400400044025876
:1029D80000000258844200241000024010464FF0C4
:1029E800000C0AE011F80C20054B9A62044BDB69D5
:1029F80013F0400FFAD00CF1010C8445F2DB70475C
:102A080000100140DFF834D0FFF72CFE0C480D49C8
:102A18000D4A002302E0D458C4500433C4188C4231
:102A2800F9D30A4A0A4C002301E013600432A24297
:102A3800FBD305F091FBFFF78DFD704700000824DC
:102A48000000002464080024849800086408002416
:102A580068440024FEE70000104B1B780BB90120E6
:102A6800704710B504464FF47A70B0FBF3F30C4A84
:102A78001068B0FBF3F000F0C7F868B90F2C01D963
:102A880001200AE0002221464FF0FF3000F078F8DC
:102A9800044B1C60002000E0012010BD1800002439
:102AA800100000241C00002410B5032000F056F884
:102AB80002F0E4F90F498B69C3F303230E4AD35C90
:102AC80003F01F03D8408B6903F00F03D35C03F0B6
:102AD8001F0320FA03F3094A1360094B18600F20FB
:102AE800FFF7BAFF10B10124204610BD0446FFF7D6
:102AF80047FDF9E700440258F8970008140000243D
:102B080010000024034B1B78034A11680B44136020
:102B1800704700BF180000241C440024014B1868AB
:102B2800704700BF1C44002438B50446FFF7F6FF81
:102B38000546B4F1FF3F02D0044B1B781C44FFF755
:102B4800EDFF401BA042FAD338BD00BF1800002497
:102B5800014B1868000C70470010005C0649CB68F0
:102B680023F4E0631B041B0C000200F4E060034341
:102B7800024A1A43CA60704700ED00E00000FA05F7
:102B880000B5174BDB68C3F30223C3F1070CBCF194
:102B9800040F28BF4FF0040C03F1040EBEF1060F1A
:102BA80014D9033B4FF0FF3E0EFA0CFC21EA0C014E
:102BB80099400EFA03F322EA03031943002807DBBE
:102BC8000901C9B2074B19545DF804FB0023E9E772
:102BD80000F00F000901C9B2034B1954F4E700BF14
:102BE80000ED00E000E400E014ED00E0002807DB61
:102BF80000F01F02400901239340024A42F82030A6
:102C0800704700BF00E100E00138B0F1807F0BD2CF
:102C18004FF0E0235861054AF02182F82310002084
:102C2800986107221A6170470120704700ED00E0A3
:102C3800F0B4876D0468664E664DAC4218BFB44266
:102C480042D01835AC423FD01835AC423CD018358C
:102C5800AC4239D01835AC4236D01835AC4233D0F6
:102C68001835AC4230D005F55675AC422CD0183525
:102C7800AC4229D01835AC4226D01835AC4223D006
:102C88001835AC4220D01835AC421DD01835AC42AE
:102C98001AD01835AC4217D04F4DAC4214D0143569
:102CA800AC4211D01435AC420ED01435AC420BD026
:102CB8001435AC4208D01435AC4205D01435AC42BA
:102CC80002D01435AC4207D1446E856E6560C46E7F
:102CD80014B1046F456F656004683D4E3D4DAC42CC
:102CE80018BFB44252D01835AC424FD01835AC4258
:102CF8004CD01835AC4249D01835AC4246D01835BE
:102D0800AC4243D01835AC4240D005F55675AC42BC
:102D18003CD01835AC4239D01835AC4236D01835CD
:102D2800AC4233D01835AC4230D01835AC422DD037
:102D38001835AC422AD01835AC4227D0264E274D3C
:102D4800AC4218BFB44211D0254DAC420ED0143558
:102D5800AC420BD01435AC4208D01435AC4205D087
:102D68001435AC4202D01435AC4224D1C46D04F001
:102D78001F050124AC407C60046863608368402BB5
:102D880020D0036899600368DA6014E0C46D04F029
:102D98001F0C3F2404FA0CF4BC6005682C6824F46A
:102DA80080242C60046863608368402B05D0036826
:102DB80099600368DA60F0BC704703689A6003683A
:102DC800D960F8E703689A600368D960F3E700BF41
:102DD8001000024028000240085402581C540258AF
:102DE8003054025803682749274A934218BF8B4238
:102DF8002FD0183293422CD01832934229D018324F
:102E0800934226D01832934223D01832934220D0CE
:102E1800183293421DD002F55672934219D01832D7
:102E2800934216D01832934213D01832934210D0DE
:102E3800183293420DD0183293420AD01832934276
:102E480007D01832934204D023F0FF038365806DC6
:102E5800704710B4D9B210390C4AA2FB0142C2F330
:102E680002120B4CA25CC2655F2906D9094A1A40B6
:102E780004328265806D10BC7047064A1A4082652C
:102E8800F8E700BF1000024028000240ABAAAAAA37
:102E98000898000800FCFFFF83699BB9836A012B2F
:102EA8000AD0022B02D00BB100207047C36A13F07E
:102EB800807F2AD100207047C36AB3F1C07F26D033
:102EC80000207047B3F5005F0AD0836A022B26D929
:102ED800032B26D1C36A13F0807F24D100207047CA
:102EE800836A032B03D8DFE803F01404140A0020D4
:102EF8007047C36A13F0807F0DD100207047C36A02
:102F0800B3F1C07F09D0002070470120704701202D
:102F18007047012070470120704701207047012049
:102F2800704700207047012070470000036822495D
:102F3800224A934218BF8B4228D01432934225D09C
:102F48001432934222D0143293421FD01432934247
:102F58001CD01432934219D01432934216D0DAB2EC
:102F6800103A1749A1FB0212120916491944A82957
:102F78001FD9154B13449B000366144B436602F09C
:102F88001F02012303FA02F282667047DBB2083B94
:102F98000F4AA2FB03230F4A02EB131292000266A8
:102FA8000D4A4266C3F30413012202FA03F383664F
:102FB80070470832DDE700BF085402581C54025815
:102FC800ABAAAAAAF0FBFDBF00820010800802404D
:102FD800CDCCCCCC009600168058025801794A1EF8
:102FE800072A2CD830B40368154D164CA34218BFD5
:102FF800AB4218D01434A34215D01434A34212D0D3
:103008001434A3420FD01434A3420CD01434A34276
:1030180009D01434A34206D00B4B0B449B00C36663
:103028000A4B036705E00A4B0B449B00C366094B38
:103038000367012303FA02F2426730BC7047704706
:10304800085402581C5402583F820010400902409C
:103058003F9600164059025870B50446FFF75EFDCA
:10306800002C00F0B681054623685349534A934221
:1030780018BF8B420CBF0122002250D030318B4246
:103088004DD018318B424AD018318B4247D0183175
:103098008B4244D018318B4241D018318B423ED0FC
:1030A80001F556718B423AD018318B4237D018311E
:1030B8008B4234D018318B4231D018318B422ED00C
:1030C80018318B422BD018318B4228D018318B42C3
:1030D80025D03B493B4A934218BF8B4200F03181CF
:1030E800394A934200F02D811432934200F029812D
:1030F8001432934200F025811432934200F021816A
:103108001432934200F01D811432934200F0198169
:1031180040236365032384F8353001204AE0022107
:1031280084F83510002184F834107ABB274A93427A
:103138002CD01832934229D01832934226D0183214
:10314800934223D01832934220D0183293421DD094
:1031580002F55672934219D01832934216D018329B
:10316800934213D01832934210D0183293420DD0A4
:10317800183293420AD01832934207D01832934239
:1031880004D01A6822F001021A6003E01A6822F0DB
:1031980001021A6023681A6812F0010F18D0FFF7AD
:1031A800BDFC431B052BF5D920236365032384F855
:1031B8003530012070BD00BF1000024028000240D9
:1031C800085402581C540258305402584000024017
:1031D8001A6881481040A168E2680A4321690A43D5
:1031E80061690A43A1690A43E1690A43216A0A43FA
:1031F8000243616A042900F099807849086878498F
:103208000140B1F1005F11D36168A1F12905A1F175
:103218003F00032888BF052D06D9A1F147000128E2
:1032280002D94F39032901D842F480121A6026685E
:10323800756925F00705636A1D43042B08D1A36A45
:103248001D43E36A23B12046FFF726FE002872D10A
:1032580075612046FFF7C6FDE36D03F01F023F23AB
:103268009340836023685F495F4A934218BF8B424B
:1032780042D0183293423FD0183293423CD0183291
:10328800934239D01832934236D01832934233D011
:103298001832934230D002F5567293422CD018322D
:1032A800934229D01832934226D01832934223D021
:1032B8001832934220D0183293421DD018329342CC
:1032C8001AD01832934217D0484A934214D0143275
:1032D800934211D0143293420ED0143293420BD041
:1032E8001432934208D01432934205D014329342D8
:1032F80002D01432934213D12046FFF717FEA36879
:10330800802B59D0236E22791A60636EA26E5A60A0
:103318006368013B072B52D90023E3662367636781
:1033280000206065012384F8353043E7E16A206BAB
:1033380001430A4361E740236365012084F83500AF
:1033480038E7022284F83520002284F834201A68ED
:1033580027491140A268402A2CD0802A27D0002271
:10336800E06842EAD002206942EAD002606942EA93
:10337800D002A06942EAD002E06942EAD002206A9B
:1033880042EA10120A431A6022681A4B13441A4A76
:10339800A2FB03231B099B00E3652046FFF722FDE0
:1033A800E26D02F01F0101228A4042605AE74FF4A1
:1033B8008042D5E71022D3E700236360A2E72046C6
:1033C800FFF70CFEE36E00221A60236F626F5A60EB
:1033D800A6E70120EEE600BF3F8010FE0010005C6B
:1033E8000000FFFF10000240280002400854025865
:1033F8000F00FEFFF8ABFDA7CDCCCCCC002800F029
:10340800DB8010B5044603686C496D4A934218BFC7
:103418008B422FD0183293422CD01832934229D0A5
:103428001832934226D01832934223D0183293424E
:1034380020D0183293421DD002F55672934219D00B
:103448001832934216D01832934213D0183293424E
:1034580010D0183293420DD0183293420AD0183245
:10346800934207D01832934204D01A6822F001021E
:103478001A6003E01A6822F001021A6023684F49B3
:103488004F4A934218BF8B4244D01832934241D0DE
:10349800183293423ED0183293423BD018329342AE
:1034A80038D01832934235D01832934232D002F5D0
:1034B800567293422ED0183293422BD01832934230
:1034C80028D01832934225D01832934222D018328D
:1034D80093421FD0183293421CD01832934219D00D
:1034E8003849394A934218BF8B4247D0374A9342EA
:1034F80044D01432934241D0143293423ED0143215
:1035080093423BD01432934238D01432934235D090
:10351800012032E000221A6023685A6023689A600A
:103528002368DA6023681A61236821225A612046D9
:10353800FFF758FCE36D03F01F023F2393408360BD
:103548002046FFF7F3FC236E23B100221A60636E56
:10355800A26E5A606368013B072B23D90020E066FE
:1035680020676067E06320646064A064E0642065AD
:10357800606584F8350084F8340010BD00221A60B4
:1035880023685A6023689A602368DA6023681A619E
:103598002046FFF727FCE36D03F01F020123934049
:1035A8004360CDE72046FFF719FDE36E00221A605D
:1035B800236F626F5A60D1E7012070471000024004
:1035C80028000240085402581C540258305402582B
:1035D800002800F03E8170B5044690F834000128B8
:1035E80000F03981012084F8340094F83500C0B225
:1035F800012807D04FF400636365002384F8343052
:10360800012070BD022084F8350000206065206824
:10361800924E934DA84218BFB0422FD01835A842F9
:103628002CD01835A84229D01835A84226D01835EC
:10363800A84223D01835A84220D01835A8421DD05A
:1036480005F55675A84219D01835A84216D0183570
:10365800A84213D01835A84210D01835A8420DD06A
:103668001835A8420AD01835A84207D01835A842FC
:1036780004D0056825F00105056003E0056825F01C
:10368800010505602046FFF7D3FA23687349744A99
:10369800934218BF8B4238D01832934235D0183233
:1036A800934232D0183293422FD0183293422CD002
:1036B8001832934229D01832934226D002F5567216
:1036C800934222D0183293421FD0183293421CD012
:1036D8001832934219D01832934216D018329342B6
:1036E80013D01832934210D0183293420DD01A6872
:1036F80022F00E0242F00A021A60236C93B122688B
:10370800136843F0040313600CE01A6822F01E02E9
:1037180042F016021A60236C23B12268136843F042
:103728000803136023684D494D4A934218BF8B42E2
:1037380042D0183293423FD0183293423CD01832CC
:10374800934239D01832934236D01832934233D04C
:103758001832934230D002F5567293422CD0183268
:10376800934229D01832934226D01832934223D05C
:103778001832934220D0183293421DD01832934207
:103788001AD01832934217D0364A934214D01432C2
:10379800934211D0143293420ED0143293420BD07C
:1037A8001432934208D01432934205D01432934213
:1037B80002D0143293420ED1236E1A6812F4803F5D
:1037C80003D01A6842F480721A60E36E1BB11A685B
:1037D80042F480721A6023682049214A934218BF34
:1037E8008B4230D0183293422DD0183293422AD0CF
:1037F8001832934227D01832934224D01832934279
:1038080021D0183293421ED002F5567293421AD034
:103818001832934217D01832934214D01832934278
:1038280011D0183293420ED0183293420BD018326E
:10383800934208D01832934205D01A6842F0010228
:103848001A600020DDE61A6842F001021A600020C2
:10385800D7E6012070470220D3E600BF10000240DF
:10386800280002400854025870B50446FFF756F97C
:10387800002C00F09181054694F83530DBB2022B1C
:1038880006D080236365002384F83430012070BD9E
:1038980023688C498C4A934218BF8B4230D0183227
:1038A80093422DD0183293422AD01832934227D00F
:1038B8001832934224D01832934221D018329342BE
:1038C8001ED002F5567293421AD01832934217D07E
:1038D8001832934214D01832934211D018329342BE
:1038E8000ED0183293420BD01832934208D01832B7
:1038F800934205D01A6822F00E021A60266809E081
:103908001A6822F01E021A602268536923F08003A5
:103918005361266823686B496B4A934218BF8B42F0
:1039280042D0183293423FD0183293423CD01832DA
:10393800934239D01832934236D01832934233D05A
:103948001832934230D002F5567293422CD0183276
:10395800934229D01832934226D01832934223D06A
:103968001832934220D0183293421DD01832934215
:103978001AD01832934217D0544A934214D01432B2
:10398800934211D0143293420ED0143293420BD08A
:103998001432934208D01432934205D01432934221
:1039A80002D01432934204D1226E136823F4807338
:1039B800136023684349444A934218BF8B422FD06F
:1039C800183293422CD01832934229D0183293429D
:1039D80026D01832934223D01832934220D018327E
:1039E80093421DD002F55672934219D01832934271
:1039F80016D01832934213D01832934210D018328E
:103A080093420DD0183293420AD01832934207D00D
:103A18001832934204D01A6822F001021A6003E0B7
:103A28001A6822F001021A60336813F0010F0ED0F1
:103A3800FFF774F8431B052BF6D92023636503238E
:103A480084F83530002384F8343001201FE72368D8
:103A58001C491D4A934218BF8B4239D018329342F1
:103A680036D01832934233D01832934230D01832BD
:103A780093422DD0183293422AD01832934227D03D
:103A880002F55672934223D01832934220D018324E
:103A980093421DD0183293421AD01832934217D04D
:103AA8001832934214D01832934211D018329342EC
:103AB8000ED0A16DE36D03F01F02012393404B600C
:103AC8000DE000BF100002402800024008540258D0
:103AD800A16DE36D03F01F023F2393408B602368C1
:103AE8002E492F4A934218BF8B4242D01832934234
:103AF8003FD0183293423CD01832934239D0183212
:103B0800934236D01832934233D01832934230D091
:103B180002F5567293422CD01832934229D01832AB
:103B2800934226D01832934223D01832934220D0A1
:103B3800183293421DD0183293421AD01832934249
:103B480017D0184A934214D01432934211D0143229
:103B580093420ED0143293420BD01432934208D0C1
:103B68001432934205D01432934202D01432934255
:103B78000BD1636EA26E5A60E36E33B11A6822F4F9
:103B880080721A60236F626F5A60012384F835309F
:103B9800002084F834007AE6012078E6100002401C
:103BA8002800024008540258002800F0298108B56E
:103BB800024690F83530DBB2022B03D080234365F0
:103BC800012008BD0368904890498B4218BF834282
:103BD8000CBF0121002166D03030834263D01830F9
:103BE800834260D0183083425DD0183083425AD067
:103BF8001830834257D01830834254D000F556709D
:103C0800834250D0183083424DD0183083424AD076
:103C18001830834247D01830834244D0183083424A
:103C280041D0183083423ED0183083423BD01968C7
:103C380021F00E0119601368A0F5956073498B4255
:103C480018BF83426AD072498B4267D018318B42C1
:103C580064D018318B4261D018318B425ED0183154
:103C68008B425BD018318B4258D001F556718B428C
:103C780054D018318B4251D018318B424ED0183164
:103C88008B424BD018318B4248D018318B4245D0EB
:103C980018318B4242D018318B423FD0196821F03D
:103CA800010119603EE0042082F8350081BB584AC2
:103CB80093422DD0183293422AD01832934227D0FB
:103CC8001832934224D01832934221D018329342AA
:103CD8001ED002F5567293421AD01832934217D06A
:103CE8001832934214D01832934211D018329342AA
:103CF8000ED0183293420BD01832934208D01832A3
:103D0800934205D01A6822F001021A60002058E791
:103D18001A6822F001021A60002052E7196821F09F
:103D2800010119601368384838498B4218BF83422B
:103D380042D018318B423FD018318B423CD01831D9
:103D48008B4239D018318B4236D018318B4233D060
:103D580018318B4230D001F556718B422CD0183176
:103D68008B4229D018318B4226D018318B4223D070
:103D780018318B4220D018318B421DD018318B421C
:103D88001AD018318B4217D022498B4214D01431E3
:103D98008B4211D014318B420ED014318B420BD090
:103DA80014318B4208D014318B4205D014318B4228
:103DB80002D014318B4217D1116E0B6823F4807333
:103DC8000B60906DD36D03F01F0101238B4043609E
:103DD800536E916E5960D36E33B1196821F48071B6
:103DE8001960136F516F5960012382F83530002331
:103DF80082F83430136D2BB1104698470020E0E666
:103E0800012070470020DCE6100002402800024034
:103E18004000024008540258F0B583B0044600231D
:103E280001937D4B1D687D4BA3FB0535AD0A876D5E
:103E38003E68D7F800C0036879497A48834218BFBA
:103E48008B420CBF0120002061D0774A93425ED09C
:103E5800183293425BD01832934258D018329342AA
:103E680055D01832934252D0183293424FD002F5AF
:103E7800567293424BD01832934248D0183293422C
:103E880045D01832934242D0183293423FD018326C
:103E980093423CD01832934239D01832934236D0EC
:103EA8006249634A934218BF8B4212D0614A9342D7
:103EB8000FD0143293420CD01432934209D01432EA
:103EC800934206D01432934203D01432934240F006
:103ED80061821A68E16D01F01F010420884010EA30
:103EE8000C0F00F0A78212F0040F00F0A382786094
:103EF80012F4004F00F05A8212F4803F40F05082D2
:103F0800A36C002B00F046822046984742E2E26DFF
:103F180002F01F0108228A40324241D070BB424A57
:103F280093422BD01832934228D01832934225D08E
:103F38001832934222D0183293421FD0183293423B
:103F48001CD002F55672934218D01832934215D0FD
:103F58001832934212D0183293420FD0183293423B
:103F68000CD01832934209D01832934206D0183236
:103F7800934203D01A68C2F3C00202E01A68C2F37F
:103F880080026AB11A6822F004021A60E36D03F035
:103F98001F0208239340BB60636D43F00103636510
:103FA800E26D02F01F0226FA02F313F0010F47D068
:103FB80023681B481B498B4218BF83423CD01831E9
:103FC8008B4239D018318B4236D018318B4233D0DE
:103FD80018318B4230D018318B422DD018318B429A
:103FE8002AD001F556718B4226D018318B4223D046
:103FF80018318B4220D018318B421DD018318B429A
:104008001AD018318B4217D018318B4214D018317E
:104018008B4211D01B6813E010000024B5814E1BA1
:104028001000024028000240400002400854025894
:104038001C540258305402585B6913F0800F3BD16E
:10404800E36D03F01F03042202FA03F3334240D066
:104058002268964896498A4218BF824235D018315C
:104068008A4232D018318A422FD018318A422CD055
:1040780018318A4229D018318A4226D018318A420A
:1040880023D001F556718A421FD018318A421CD0BC
:1040980018318A4219D018318A4216D018318A420A
:1040A80013D018318A4210D018318A420DD01831F5
:1040B8008A420AD013680CE0012303FA02F2BA60BC
:1040C800636D43F002036365BAE7126812F0020FEA
:1040D8003DD1E36D03F01F03102202FA03F33342CC
:1040E8005FD02268714872498A4218BF824234D030
:1040F80018318A4231D018318A422ED018318A427A
:104108002BD018318A4228D018318A4225D018314C
:104118008A4222D001F556718A421ED018318A424D
:104128001BD018318A4218D018318A4215D018315C
:104138008A4212D018318A420FD018318A420CD0E4
:1041480018318A4209D01268C2F3800208E0BB60C5
:10415800636D43F004036365BBE71268C2F3C002F2
:10416800FAB1BB6023681A6812F4802F0DD01B685F
:1041780013F4002F04D1236C9BB12046984710E01C
:10418800A36C73B1204698470BE01A6812F4807F3D
:1041980003D11A6822F008021A60236C0BB120467A
:1041A8009847E36D03F01F03202202FA03F333421A
:1041B80000F0928022683D483D498A4218BF8242F9
:1041C8002ED018318A422BD018318A4228D0183183
:1041D8008A4225D018318A4222D018318A421FD00B
:1041E80018318A421CD001F556718A4218D018310C
:1041F8008A4215D018318A4212D018318A420FD01B
:1042080018318A420CD018318A4209D018318A42B2
:1042180006D018318A4203D01268C2F3400202E085
:104228001268C2F30012002A56D0BB6094F83530E9
:10423800DBB2042B0ED023681A6812F4802F39D011
:104248001B6813F4002F2CD1636C002B44D020463C
:10425800984741E02268136823F016031360226828
:10426800536923F080035361236CB3B12268136848
:1042780023F008031360E36D03F01F023F2393400C
:10428800BB60012384F83530002384F83430236D73
:10429800002B7FD0204698477CE0A36C002BE5D10B
:1042A800E9E7E36BC3B12046984715E010000240E8
:1042B800280002401A6812F4807F09D11A6822F097
:1042C80010021A60012384F83530002384F8343052
:1042D800E36B0BB120469847636D002B5AD0636D92
:1042E80013F0010F52D0042384F83530236896491F
:1042F800964A934218BF8B422FD0183293422CD043
:104308001832934229D01832934226D01832934259
:1043180023D01832934220D0183293421DD002F590
:104328005672934219D01832934216D018329342DB
:1043380013D01832934210D0183293420DD018324D
:1043480093420AD01832934207D01832934204D0CD
:104358001A6822F001021A6003E01A6822F00102CA
:104368001A60019B01330193AB4204D823681B6890
:1043780013F0010FF5D123681B6813F0010F0BD060
:10438800032384F83530002384F83430E36C0BB110
:104398002046984703B0F0BD012384F83530F2E792
:1043A800236C002BF6D020469847F3E712F0200F35
:1043B8003AD123686449654A934218BF8B422FD08B
:1043C800183293422CD01832934229D01832934293
:1043D80026D01832934223D01832934220D0183274
:1043E80093421DD002F55672934219D01832934267
:1043F80016D01832934213D01832934210D0183284
:1044080093420DD0183293420AD01832934207D003
:104418001832934204D01A6822F004021A6003E0AA
:104428001A6822F008021A60236C002BB2D02046CA
:104438009847AFE70220884010EA0C0F60D012F0CE
:10444800020F5DD0786012F4004F0ED012F4803F56
:1044580005D1636C002B9DD0204698479AE7E36B03
:10446800002B97D02046984794E712F0200F40D1B0
:1044780023683549354A934218BF8B422FD01832EA
:1044880093422CD01832934229D01832934226D026
:104498001832934223D01832934220D018329342D4
:1044A8001DD002F55672934219D01832934216D095
:1044B8001832934213D01832934210D018329342D4
:1044C8000DD0183293420AD01832934207D01832CE
:1044D800934204D01A6822F00A021A6003E01A68AC
:1044E80022F014021A60012384F83530002384F87E
:1044F8003430E36B002B3FF44DAF2046984749E733
:10450800082000FA01F111EA0C0F3FF443AF12F052
:10451800080F3FF43FAF1A6822F00E021A60E36DED
:1045280003F01F03012202FA03F37B60626584F83B
:104538003520002384F83430E36C002B3FF42AAF95
:104548002046984726E700BF100002402800024096
:10455800406D704770B582B000236EE085685E00DC
:104568000324B44025EA0405CC68B4402C43846095
:10457800446824EA0C0C4C68C4F300149C4044EAD8
:104588000C0444606CE0DD08083550F8256003F041
:1045980007044FEA840C0F2404FA0CF426EA040EEC
:1045A8000C6904FA0CF444EA0E0440F825406FE064
:1045B800092400E0002404FA0EF42C430CF1020C48
:1045C8006B4D45F82C404FF0B0442568D44325EA9C
:1045D8000206D1F804C01CF4801F01D042EA050687
:1045E8004FF0B0452E606D6804EA0506D1F804C0A6
:1045F8001CF4001F01D042EA05064FF0B0456E607A
:10460800D5F8845004EA0506D1F804C01CF4003F2C
:1046180001D042EA05064FF0B045C5F88460D5F8E8
:1046280080502C404E6816F4803F01D042EA0504C1
:104638004FF0B042C2F8804001330A6832FA03F4FE
:1046480000F093804FF0010C0CFA03FC1CEA020204
:10465800F2D04C6804F00304013C012C7FF67EAFD5
:104668004C6804F00304032C0CD0C4685D004FF0C0
:10467800030C0CFA05FC24EA0C0C8C68AC4044EAE8
:104688000C04C4604C6804F00304022C3FF47BAFB4
:1046980004684FEA430E4FF0030C0CFA0EFC24EAB0
:1046A8000C0C4C6804F0030404FA0EF444EA0C04FD
:1046B80004604C6814F4403FBED02E4CD4F8F4503B
:1046C80045F00205C4F8F450D4F8F44004F00204AC
:1046D8000194019C4FEA930C0CF10205244C54F808
:1046E800255003F003044FEA840E0F2404FA0EF455
:1046F80025EA0405204CA0423FF45CAF04F5806431
:10470800A04222D004F58064A04220D004F5806441
:10471800A0421ED004F58064A0421CD004F5806439
:10472800A0421AD004F58064A04218D004F5806431
:10473800A04216D004F58064A04214D004F5806429
:10474800A0423FF435AF0A2435E7012433E70224B9
:1047580031E703242FE704242DE705242BE706245B
:1047680029E7072427E7082425E702B070BD00BF22
:104778000004005800440258000002580369194216
:1047880001D001207047002070470AB1816170474D
:1047980009048161704708B54FF0B043D3F88830F9
:1047A800034200D108BD4FF0B043C3F88800FDF7BD
:1047B80065FBF7E7134BDB6813F0040F07D1114BC8
:1047C800DB6803F0070383421AD00120704710B555
:1047D8000C4AD36823F007031843D060FEF79EF90C
:1047E8000446084B5B6813F4005F07D1FEF796F99F
:1047F800001BB0F57A7FF4D9012000E0002010BD3D
:104808000020704700480258002800F0188338B587
:104818000446036813F0010F25D0944A136903F086
:104828003803926A102B15D0182B0FD06368B3F594
:10483800803F3FD0002B53D18C4B1A6822F4803232
:104848001A601A6822F480221A6038E002F0030223
:10485800022AEBD1854B1B6813F4003F03D0636831
:10486800002B00F0EE82236813F0020F00F0A18005
:104878007E4A1369926A13F038035AD0182B55D020
:10488800E368002B00F0DE8078490A6822F01902FC
:1048980013430B60FEF742F90546744B1B6813F08F
:1048A800040F40F0AD80FEF739F9401B0228F4D917
:1048B8000320CDE26D4A136843F4803313606368C4
:1048C8002BB3FEF72BF90546684B1B6813F4003F22
:1048D800C9D1FEF723F9401B6428F5D90320B7E2B4
:1048E800B3F5A02F09D0614B1A6822F480321A6000
:1048F8001A6822F480221A60E1E75C4B1A6842F4D5
:1049080080221A601A6842F480321A60D7E7FEF7EC
:1049180005F90546554B1B6813F4003FA3D0FEF775
:10492800FDF8401B6428F5D9032091E212F0030F2B
:10493800A6D14E4B1B6813F0040F03D0E368002B7D
:1049480000F08182494A136823F01903E1680B4398
:104958001360FEF7E3F80546444B1B6813F0040F99
:1049680006D1FEF7DBF8401B0228F5D903206FE2D9
:10497800FEF7EEF841F20303984212D82269402A62
:1049880007D03A494B6823F47C3343EA02334B603F
:104998000FE0364A536823F47C3343F40033536002
:1049A80007E0324A536823F0FE43216943EA016372
:1049B8005360236813F0100F00F088802B4A1369A6
:1049C80003F03803926A082B56D0182B50D0E369AD
:1049D800002B00F0B880254A136843F08003136069
:1049E800FEF79CF80546214B1B6813F4807F40F0C6
:1049F8008880FEF793F8401B0228F4D9032027E2A9
:104A0800FEF7A6F841F20303984212D82269402A19
:104A180007D016494B6823F47C3343EA02334B60D2
:104A2800C7E7124A536823F47C3343F400335360D6
:104A3800BFE70E4A536823F0FE43216943EA016346
:104A48005360B6E7094A136823F001031360FEF7C1
:104A580065F80546054B1B6813F0040FA9D0FEF74F
:104A68005DF8401B0228F5D90320F1E10044025803
:104A780002F00302012AAAD1A14B1B6813F4807F1C
:104A880003D0E369802B40F0E081FEF761F841F242
:104A98000303984212D8226A202A07D098494B6803
:104AA80023F0F84343EA82634B600FE0944A53686B
:104AB80023F0F84343F08043536007E0904AD368FB
:104AC80023F07C53216A43EA0163D360236813F01F
:104AD800080F60D06369002B49D0894A536F43F0AF
:104AE80001035367FEF71AF80546854B5B6F13F011
:104AF800020F50D1FEF712F8401B0228F5D9032007
:104B0800A6E1FEF725F841F20303984212D8226A7B
:104B1800202A07D07A494B6823F0F84343EA826396
:104B28004B60D3E7764A536823F0F84343F0804359
:104B38005360CBE7724AD36823F07C53216A43EA77
:104B48000163D360C2E76E4A136823F080031360E1
:104B5800FDF7E4FF05466A4B1B6813F4807FB5D068
:104B6800FDF7DCFF401B0228F5D9032070E1644AF9
:104B7800536F23F001035367FDF7D0FF0546604BE1
:104B88005B6F13F0020F06D0FDF7C8FF401B022829
:104B9800F5D903205CE1236813F0200F29D0A3691D
:104BA8009BB1574A136843F480531360FDF7B6FF6F
:104BB8000546534B1B6813F4005F1AD1FDF7AEFF8F
:104BC800401B0228F5D9032042E14D4A136823F41B
:104BD80080531360FDF7A2FF0546494B1B6813F489
:104BE800005F06D0FDF79AFF401B0228F5D9032085
:104BF8002EE1236813F0040F21D1636A002B00F023
:104C080026813F4A126902F03802182A00F0EE8025
:104C1800022B79D03A4A136823F080731360FDF7AA
:104C28007DFF0446364B1B6813F0007F00F0DC80E4
:104C3800FDF774FF001B0228F4D9032008E1314A6C
:104C4800136843F480731360FDF768FF05462D4B26
:104C58001B6813F4807F06D1FDF760FF401B6428B2
:104C6800F5D90320F4E0A368012B0AD00BBB244B31
:104C78001A6F22F001021A671A6F22F004021A67EB
:104C880004E01F4A136F43F001031367A36833B3AB
:104C9800FDF744FF05461A4B1B6F13F0020FACD10A
:104CA800FDF73CFF401B41F288339842F3D90320BB
:104CB800CEE0052B09D0124B1A6F22F001021A67B9
:104CC8001A6F22F004021A67E0E70D4B1A6F42F0E0
:104CD80004021A671A6F42F001021A67D6E7FDF755
:104CE8001DFF0546064B1B6F13F0020F85D0FDF71D
:104CF80015FF401B41F288339842F3D90320A7E0FF
:104D08000044025800480258594A136823F0807337
:104D18001360FDF703FF0546554B1B6813F0007F32
:104D280006D0FDF7FBFE401B0228F5D903208FE0D3
:104D38004F4B996A4F4A0A40A16AE06A41EA00115A
:104D48000A439A62226B013AC2F30802616B013985
:104D5800490289B20A43A16B0139090401F4FE0131
:104D68000A43E16B0139090601F0FE410A431A635F
:104D7800DA6A22F00102DA62596B3F4A0A40A16CF2
:104D880042EAC1025A63DA6A22F00C02216C0A4331
:104D9800DA62DA6A22F00202616C0A43DA62DA6ADB
:104DA80042F48032DA62DA6A42F40032DA62DA6AAB
:104DB80042F48022DA62DA6A42F00102DA621A68A0
:104DC80042F080721A60FDF7A9FE0446284B1B6862
:104DD80013F0007F06D1FDF7A1FE001B0228F5D9CC
:104DE800032035E0002033E0002031E0204A916ABA
:104DF800106B012B2DD001F00303A26A93422AD134
:104E0800C1F30511E36A994227D1C0F30802236B65
:104E1800013B9A4223D1C0F34622636B013B9A427D
:104E28001FD1C0F30642A36B013B9A421BD1C0F3CA
:104E38000660E36B013B984217D1002008E001208F
:104E48007047012004E0012002E0012000E000207A
:104E580038BD0120FCE70120FAE70120F8E701202E
:104E6800F6E70120F4E70120F2E70120F0E700BFB0
:104E7800004402580CFCFFFF0700FFFFF8B57E4B0B
:104E88001B6903F03803102B00F0F280182B10D0A8
:104E980013B17A4C2046F8BD774B1B6813F0200FEE
:104EA80000F0E880744B1868C0F3C100744CC4402B
:104EB800F0E7714B9D6A05F003059C6AC4F305147D
:104EC800D86A00F001005B6BC3F3CC0303FB00F06E
:104ED800FBF7A2FF0646002CDCD0012D76D0022D70
:104EE80000F0A4800DB32046FBF796FF0146654805
:104EF800FCF79EF80446604B186BC0F30800FBF7FC
:104F08008BFF05464FF064513046FBF7DDFF014645
:104F18002846FBF7D1FE4FF07E51FBF7CDFE014648
:104F28002046FBF7D1FF044671E0534B1B6813F092
:104F3800200F29D0504F3B68C3F3C1035048D840D5
:104F4800FBF76AFF05462046FBF766FF0146284641
:104F5800FCF76EF80446386BC0F30800FBF75CFFFB
:104F680005464FF064513046FBF7AEFF0146284630
:104F7800FBF7A2FE4FF07E51FBF79EFE014620464E
:104F8800FBF7A2FF044642E02046FBF745FF014637
:104F98003D48FCF74DF80446374B186BC0F3080042
:104FA800FBF73AFF05464FF064513046FBF78CFF9C
:104FB80001462846FBF780FE4FF07E51FBF77CFE4A
:104FC80001462046FBF780FF044620E02046FBF719
:104FD80023FF01462B48FCF72BF80446264B186B99
:104FE800C0F30800FBF718FF05464FF06451304640
:104FF800FBF76AFF01462846FBF75EFE4FF07E513D
:10500800FBF75AFE01462046FBF75EFF04461A4BA3
:105018001B6BC3F34623581CFBF7FEFE01462046D4
:10502800FCF706F8FCF7A0F8044633E72046FBF740
:10503800F3FE01461548FBF7FBFF04460E4B186BC1
:10504800C0F30800FBF7E8FE05464FF06451304610
:10505800FBF73AFF01462846FBF72EFE4FF07E513C
:10506800FBF72AFE01462046FBF72EFF0446CEE753
:10507800074C0FE7024C0DE70044025800093D00B9
:105088000090D0030024744A0024744C20BCBE4B0A
:1050980040787D01002800F0328170B50D46044645
:1050A8009B4B1B6803F00F038B420BD2984A136883
:1050B80023F00F030B431360136803F00F038B42B5
:1050C80040F01F81236813F0040F0CD02269914B24
:1050D8009B6903F070039A4205D98E498B6923F0C6
:1050E80070031A438A61236813F0080F0CD06269B1
:1050F800884BDB6903F070039A4205D98549CB696F
:1051080023F070031A43CA61236813F0100F0CD000
:10511800A269804BDB6903F4E0639A4205D97D49B3
:10512800CB6923F4E0631A43CA61236813F0200FA4
:105138000CD0E269774B1B6A03F070039A4205D9D9
:1051480074490B6A23F070031A430A62236813F048
:10515800020F0CD0E2686F4B9B6903F00F039A4271
:1051680005D96C498B6923F00F031A438A612368B8
:1051780013F0010F41D0674A936923F47063A16863
:105188000B4393616368022B0AD0032B27D0012BB2
:105198002CD0604A126812F0040F06D10120ADE04D
:1051A800126812F4003F00F0AE805A490A6922F0F2
:1051B800070213430B61FDF7B1FC0646554B1B690B
:1051C80003F038036268B3EBC20F16D0FDF7A6FCF4
:1051D800801B41F288339842F0D903208EE04D4A73
:1051E800126812F0007FE0D1012087E0494A126876
:1051F80012F4807FD9D1012080E0236813F0020FD8
:105208000CD0E268434B9B6903F00F039A4205D226
:1052180040498B6923F00F031A438A613C4B1B6892
:1052280003F00F03AB420AD9394A136823F00F037E
:105238002B431360136803F00F03AB4265D1236857
:1052480013F0040F0CD02269324B9B6903F07003F2
:105258009A4205D22F498B6923F070031A438A6159
:10526800236813F0080F0CD062692A4BDB6903F03E
:1052780070039A4205D22749CB6923F070031A4379
:10528800CA61236813F0100F0CD0A269214BDB69A7
:1052980003F4E0639A4205D21E49CB6923F4E06324
:1052A8001A43CA61236813F0200F0CD0E269194B26
:1052B8001B6A03F070039A4205D216490B6A23F061
:1052C80070031A430A62FFF7D9FD12498B69C3F3C9
:1052D8000323114AD35C03F01F03D8408B6903F002
:1052E8000F03D35C03F01F0320FA03F30B4A136088
:1052F8000B4B18600B4B1868FDF7AEFB70BD012017
:1053080070470120FAE70120F8E70120F6E700BF1F
:105318000020005200440258F897000814000024A6
:10532800100000241C00002408B5FFF7A7FD0B4A55
:105338009369C3F303230A49CB5C03F01F0320FAE4
:1053480003F3926902F00F02885C00F01F0023FA51
:1053580000F0044A1060044A136008BD0044025873
:10536800F8970008140000241000002408B5FFF77F
:10537800DBFF054BDB69C3F30213044AD35C03F07C
:105388001F03D84008BD00BF00440258F897000822
:1053980008B5FFF7C9FF054BDB69C3F30223044ACD
:1053A800D35C03F01F03D84008BD00BF0044025877
:1053B800F8970008404B9B6A03F00303032B79D04E
:1053C80070B505460E463C4A136823F080631360A7
:1053D800FDF7A4FB0446384B1B6813F0006F06D09A
:1053E800FDF79CFB031B022BF5D9032070BD324B44
:1053F8009A6A22F47C32296842EA01329A626A681F
:10540800013AC2F30802A9680139490289B20A437C
:10541800E9680139090401F4FE010A4329690139DF
:10542800090601F0FE410A439A63DA6A22F0C002D3
:1054380069690A43DA62DA6A22F02002A9690A4332
:10544800DA62DA6A22F01002DA62D96B1B4A0A4081
:10545800E96942EAC102DA63DA6A42F01002DA6202
:10546800C6B91A46DB6A43F40023D362124A1368AA
:1054780043F080631360FDF751FB04460E4B1B6835
:1054880013F0006F14D1FDF749FB001B0228F5D972
:105498000320ABE7012E05D0074AD36A43F4001373
:1054A800D362E3E7044AD36A43F48013D362DDE7A7
:1054B80000209BE701207047004402580700FFFFC7
:1054C800404B9B6A03F00303032B79D070B5054664
:1054D8000E463C4A136823F080531360FDF71EFB09
:1054E8000446384B1B6813F0005F06D0FDF716FB27
:1054F800031B022BF5D9032070BD324B9A6A22F0A8
:105508007C72296842EA01529A626A68013AC2F3D7
:105518000802A9680139490289B20A43E9680139D0
:10552800090401F4FE010A4329690139090601F059
:10553800FE410A431A64DA6A22F4406269690A433E
:10554800DA62DA6A22F40072A9690A43DA62DA6A6C
:1055580022F48072DA62596C1B4A0A40E96942EA0D
:10556800C1025A64DA6A42F48072DA62C6B91A462B
:10557800DB6A43F48003D362124A136843F0805312
:105588001360FDF7CBFA04460E4B1B6813F0005F5F
:1055980014D1FDF7C3FA001B0228F5D90320ABE7A5
:1055A800012E05D0074AD36A43F08073D362E3E73C
:1055B800044AD36A43F40003D362DDE700209BE783
:1055C80001207047004402580700FFFFF8B5044661
:1055D800036813F0006F30D0436EB3F5001F26D078
:1055E8000ED8EBB1B3F5801F07D102210430FFF7C5
:1055F800E1FE054645B12E4621E0012635461EE06E
:10560800B3F5401F09D10025954A136D23F44013C3
:10561800616E0B431365002611E0012635460EE046
:105628008F4AD36A43F40033D3620025ECE70221A2
:105638002430FFF745FF0546DCE70026354623689A
:1056480013F4807F14D0636D042B30D8DFE803F0A7
:10565800032228080800824AD36A43F40033D3623D
:1056680045BB7F4A136D23F00703616D0B43136538
:10567800236813F4007F2FD0A36D802B49D01ED848
:10568800002B40D0402B17D10021201DFFF792FEA0
:10569800054619E00021201DFFF78CFE0546DFE7CF
:1056A800002104F12400FFF70BFF0546D8E7012687
:1056B8003546DDE72E46DBE7012635460CE0C02BF4
:1056C80002D0B3F5807F1BD155BB654A136D23F417
:1056D800E073A16D0B431365236813F4806F45D005
:1056E800D4F8A430B3F5800F38D01ED883B3B3F5FF
:1056F800001F17D10021201DFFF75CFE05461AE0A8
:1057080001263546E8E7564AD36A43F40033D362A4
:10571800DAE7002104F12400FFF7D2FE0546D3E7BB
:105728002E46D9E70126354620E0B3F5C00F02D052
:10573800B3F5000F09D1C5B9494A936D23F4600345
:10574800D4F8A4100B43936510E0012635460DE00C
:10575800434AD36A43F40033D362ECE7002104F1EF
:105768002400FFF7ADFE0546E5E72E46236813F44F
:10577800006F23D0D4F8A830B3F1007F41D00DD802
:10578800002B38D0B3F1807F05D10021201DFFF711
:1057980011FE054608E0012635460FE0B3F1407FCB
:1057A80002D0B3F1806F23D1002D31D12C4A936DF3
:1057B80023F0E063D4F8A8100B439365236813F033
:1057C800007F2ED0A36C202B3FD026D833B1102BCE
:1057D80020D1234AD36A43F40033D362002D3AD14F
:1057E8001F4AD36C23F03003A16C0B43D36418E039
:1057F80001263546E2E71A4AD36A43F40033D362F6
:10580800D2E7002104F12400FFF75AFE0546CBE752
:105818002E46D3E70126354603E0302BDED001269D
:105828003546236813F4805F2BD0E36DB3F5005F32
:105838004CD017D8002B43D0B3F5805F0DD1002191
:10584800201DFFF7B7FD054612E00221201DFFF7D6
:10585800B1FD0546C2E72E46E3E70126354610E0CE
:1058680000440258B3F5405F02D0B3F5804F24D10D
:10587800002D32D1754A136D23F4E043E16D0B43DB
:105888001365236813F4005F37D0236EB3F5003F28
:1058980051D027D83BB1B3F5803F20D10121201D3D
:1058A800FFF788FD0546002D4CD1684A136D23F497
:1058B800E023216E0B4313651FE001263546E0E720
:1058C800624AD36A43F40033D362D1E7002104F17A
:1058D8002400FFF7F5FD0546CAE72E46D1E7012665
:1058E80035460AE0B3F5802FDDD0B3F5A02FDAD026
:1058F800B3F5403FD7D001263546236813F4804FCF
:1059080030D0D4F8AC30B3F1005F44D01FD83BB1ED
:10591800B3F1805F18D10121201DFFF74BFD05462B
:10592800002D3FD1494A936D23F0E043D4F8AC10E1
:105938000B43936516E0012104F12400FFF7C0FD35
:105948000546B0E72E46D8E7012635460AE0B3F10A
:10595800804FE5D0B3F1A04FE2D0B3F1405FDFD084
:1059680001263546236813F4004F09D0E36EB3F1DE
:10597800805F19D0B3F1005F24D0D3B1012635463A
:10598800236813F0807F32D0636C032B59D8DFE88B
:1059980003F026215226012104F12400FFF790FD8F
:1059A8000546BDE72E46DDE7284AD36A43F40033AF
:1059B800D3626DB9254A136D23F04053E16E0B4352
:1059C8001365DDE70121201DFFF7F4FC0546F0E72C
:1059D8002E46D5E71D4AD36A43F40033D3629DBBF4
:1059E8001A4AD36C23F00303616C0B43D364236816
:1059F80013F4800F2CD1236813F0010F00F0A3805B
:105A0800A36F282B00F29D80DFE803F08B9B9B9B04
:105A18009B9B9B9B869B9B9B9B9B9B9B949B9B9BEA
:105A28009B9B9B9B8B9B9B9B9B9B9B9B8B9B9B9BDE
:105A38009B9B9B9B8B000221201DFFF7BBFC05460F
:105A4800CDE701263546D2E72E46D0E70044025876
:105A58008F4A136843F480731360FDF75FF80746B5
:105A68008B4B1B6813F4807F05D1FDF757F8C01BDB
:105A78006428F5D90325002D4AD1864B1B6FD4F82D
:105A8800B020534013F4407F0CD0824B1A6F22F49D
:105A98004072196F41F480311967196F21F4803110
:105AA80019671A67D4F8B030B3F5807F15D08DBB6D
:105AB800D4F8B03003F44072B2F5407F1ED0754A76
:105AC800136923F47C53136172490B6FD4F8B02027
:105AD800C2F30B0213430B678DE7FDF71FF8074668
:105AE8006C4B1B6F13F0020FE1D1FDF717F8C01BC9
:105AF80041F288339842F3D90325D8E7654802690B
:105B080022F47C52644901EA131313430361DBE76F
:105B18002E4670E72E466EE70121201DFFF74AFC4E
:105B28000546E5B95B4A536D23F03803A16F0B4373
:105B3800536508E0012104F12400FFF7C1FC054684
:105B4800EFE701263546236813F0020F16D0636F7E
:105B5800052B27D8DFE803F00A051F0A0A0A2E4694
:105B6800F1E70121201DFFF725FC0546EDB9494A5B
:105B7800536D23F00703616F0B435365236813F0DC
:105B8800040F22D0D4F89030052B43D8DFE803F077
:105B9800140F3B141414012104F12400FFF790FCA6
:105BA8000546E3E701263546E8E72E46E6E7012104
:105BB800201DFFF7FFFB05467DBB364A936D23F09A
:105BC8000703D4F890100B439365236813F0200F54
:105BD80033D0D4F88C30B3F1005F4CD022D83BB12D
:105BE800B3F1805F1BD10021201DFFF7E3FB0546C1
:105BF800002D47D1274A536D23F0E043D4F88C1089
:105C08000B43536519E0012104F12400FFF758FC08
:105C18000546D1E701263546D7E72E46D5E70126C2
:105C280035460AE0B3F1804FE2D0B3F1A04FDFD0A0
:105C3800B3F1405FDCD001263546236813F0400FEE
:105C480037D0D4F89830B3F5006F52D026D83BB18E
:105C5800B3F5806F18D10021201DFFF7ABFB054677
:105C6800002D4DD10B4A936D23F4E053D4F89810CE
:105C78000B4393651DE0022104F12400FFF720FC8B
:105C88000546B5E72E46D8E70126354611E000BFA0
:105C98000048025800440258CFFFFF00B3F5805F68
:105CA800DED0B3F5A05FDBD0B3F5406FD8D00126C6
:105CB8003546236813F0800F32D0D4F89C30B3F502
:105CC800804F00F09D8020D83BB1B3F5005F19D11B
:105CD8000021201DFFF76EFB0546002D40F0978040
:105CE800A54A936D23F46043D4F89C100B43936545
:105CF80016E0022104F12400FFF7E2FB0546AFE7B6
:105D08002E46D6E7012635460AE0B3F5004FE4D023
:105D1800B3F5204FE1D0B3F5C04FDED001263546AC
:105D2800236813F0080F0CD0D4F88030B3F5805FE7
:105D38006FD0914A536D23F44053D4F880100B432D
:105D48005365236813F0100F0CD0D4F89430B3F5D2
:105D5800807F67D0884A936D23F44073D4F89410F9
:105D68000B439365236813F4002F0BD0D4F8A030AD
:105D7800B3F5803F6ED0B3F5003F61D0002B5AD009
:105D880001263546236813F4802F0CD0D4F88430CC
:105D9800B3F5001F76D0B3F5401F69D0B3F5801F67
:105DA80061D001263546236813F4803F07D0E36CA1
:105DB800002B70D0B3F5803F7BD001263546236891
:105DC80013F0005F7DD1236813F4003F00F0868054
:105DD800E36FB3F5807F00F0C6807CD9B3F5007F10
:105DE80003D0B3F5407F40F0BC80002D40F0C18067
:105DF800614A536D23F44073E16F0B4353656DE0C3
:105E0800022104F12400FFF75BFB054665E72E46F7
:105E180086E7022104F12400FFF752FB002888D00E
:105E2800012686E7022104F12400FFF749FB002838
:105E380090D001268EE70021201DFFF7BBFA05460A
:105E48007DB94D4A936D23F44033D4F8A0100B4329
:105E5800936597E7022104F12400FFF731FB05461B
:105E6800EEE72E468EE7444AD36A43F40033D36202
:105E78007DB9414A536D23F44013D4F884100B4381
:105E8800536590E7012104F12400FFF719FB05464B
:105E9800EEE72E4687E7384AD36A43F40033D362E5
:105EA8006DB9354AD36C23F48033E16C0B43D3646A
:105EB80085E70221201DFFF77DFA0546F0E72E460B
:105EC8007DE7022104F12400FFF7FAFA00283FF4E5
:105ED8007AAF012677E7002B87D00126236813F4D1
:105EE800801F06D0244A136D23F00043216F0B4313
:105EF8001365236813F0805F07D01F4A136923F4E2
:105F08008043D4F8B4100B431361236813F4001FC3
:105F180006D0194A136D23F08073A16E0B431365E5
:105F2800236813F0804F09D0134B1A6922F40042FA
:105F38001A611A69D4F8B8100A431A612368002B49
:105F48001CDB236813F4000F07D00B4A536D23F4AE
:105F58004003D4F888100B43536506B10126304638
:105F6800F8BD0126BAE7044AD36A43F40033D36282
:105F78003BE72E46B2E700BF00440258034AD36C01
:105F880023F04053216D0B43D364DAE700440258F1
:105F980008B5FFF7C9F9054B1B6AC3F30213044A96
:105FA800D35C03F01F03D84008BD00BF004402586B
:105FB800F89700082DE9F0410446864B9D6A9E6AD1
:105FC800C6F30536D86AC0F30010DB6BC3F3CC0305
:105FD80003FB00F0FAF720FF002E00F0F58005F033
:105FE80003050746012D79D0022D00F0CB800DB3B3
:105FF8003046FAF711FF01467748FBF719F80546CE
:10600800744B986BC0F30800FAF706FF06464FF08A
:1060180064513846FAF758FF01463046FAF74CFE05
:106028004FF07E51FAF748FE01462846FAF74CFF32
:10603800054674E0674B1B6813F0200F2CD0DFF87F
:106048009481D8F80030C3F3C1036448D840FAF704
:10605800E3FE05463046FAF7DFFE01462846FAF722
:10606800E7FF0546D8F83800C0F30800FAF7D4FE71
:1060780006464FF064513846FAF726FF0146304687
:10608800FAF71AFE4FF07E51FAF716FE0146284637
:10609800FAF71AFF054642E03046FAF7BDFE014618
:1060A8004F48FAF7C5FF05464A4B986BC0F30800FE
:1060B800FAF7B2FE06464FF064513846FAF704FF85
:1060C80001463046FAF7F8FD4FF07E51FAF7F4FD35
:1060D80001462846FAF7F8FE054620E03046FAF76A
:1060E8009BFE01463C48FAF7A3FF0546394B986BDF
:1060F800C0F30800FAF790FE06464FF064513846A0
:10610800FAF7E2FE01463046FAF7D6FD4FF07E5127
:10611800FAF7D2FD01462846FAF7D6FE05462D4E77
:10612800B06BC0F34620FAF777FE4FF07E51FAF7CE
:10613800C3FD01462846FAF77BFFFBF715F82060F8
:10614800B06BC0F30640FAF767FE4FF07E51FAF7DE
:10615800B3FD01462846FAF76BFFFBF705F86060C8
:10616800B06BC0F30660FAF757FE4FF07E51FAF7AE
:10617800A3FD01462846FAF75BFFFAF7F5FFA06092
:10618800BDE8F0813046FAF747FE01461548FAF7B0
:106198004FFF05460F4B986BC0F30800FAF73CFE1B
:1061A80006464FF064513846FAF78EFE01463046EF
:1061B800FAF782FD4FF07E51FAF77EFD0146284638
:1061C800FAF782FE0546AAE7002323606360A3600E
:1061D800D6E700BF004402580024744A0090D00358
:1061E8000024744C20BCBE4B2DE9F0410446864B7C
:1061F8009D6A9E6AC6F30556D86AC0F300205B6C98
:10620800C3F3CC0303FB00F0FAF706FE002E00F000
:10621800F58005F003050746012D79D0022D00F021
:10622800CB800DB33046FAF7F7FD01467748FAF709
:10623800FFFE0546744B186CC0F30800FAF7ECFD36
:1062480006464FF064513846FAF73EFE014630469E
:10625800FAF732FD4FF07E51FAF72EFD0146284637
:10626800FAF732FE054674E0674B1B6813F0200FFF
:106278002CD0DFF89481D8F80030C3F3C103644808
:10628800D840FAF7C9FD05463046FAF7C5FD01467C
:106298002846FAF7CDFE0546D8F84000C0F30800B6
:1062A800FAF7BAFD06464FF064513846FAF70CFE85
:1062B80001463046FAF700FD4FF07E51FAF7FCFC34
:1062C80001462846FAF700FE054642E03046FAF74E
:1062D800A3FD01464F48FAF7ABFE05464A4B186C3A
:1062E800C0F30800FAF798FD06464FF064513846A7
:1062F800FAF7EAFD01463046FAF7DEFC4FF07E5128
:10630800FAF7DAFC01462846FAF7DEFD054620E0F2
:106318003046FAF781FD01463C48FAF789FE054602
:10632800394B186CC0F30800FAF776FD06464FF0B3
:1063380064513846FAF7C8FD01463046FAF7BCFC06
:106348004FF07E51FAF7B8FC01462846FAF7BCFD33
:1063580005462D4E306CC0F34620FAF75DFD4FF030
:106368007E51FAF7A9FC01462846FAF761FEFAF7CA
:10637800FBFE2060306CC0F30640FAF74DFD4FF08D
:106388007E51FAF799FC01462846FAF751FEFAF7CA
:10639800EBFE6060306CC0F30660FAF73DFD4FF02D
:1063A8007E51FAF789FC01462846FAF741FEFAF7CA
:1063B800DBFEA060BDE8F0813046FAF72DFD01460E
:1063C8001548FAF735FE05460F4B186CC0F3080060
:1063D800FAF722FD06464FF064513846FAF774FD85
:1063E80001463046FAF768FC4FF07E51FAF764FC34
:1063F80001462846FAF768FD0546AAE70023236008
:106408006360A360D6E700BF004402580024744AC2
:106418000090D0030024744C20BCBE4B10B4036A17
:10642800046A24F001040462846924F0F00C4CEA44
:10643800021223F00A030B438261036210BC704707
:1064480010B4046A24F0100404628469036A24F412
:10645800704C4CEA023223F0A00343EA0113826134
:10646800036210BC704700008268034B13400B4363
:1064780043F00703836070478FFFCFFF90F83D30EC
:10648800DBB2012B35D1022380F83D3003681B4A6B
:10649800B3F1804F18BF93421DD0A2F57C429342BE
:1064A80019D002F58062934215D002F580629342BA
:1064B80011D002F5784293420DD0A2F56C42934276
:1064C80009D002F59432934205D01A6842F00102CD
:1064D8001A60002070479968094A0A40062A18BFBE
:1064E800B2F5803F07D01A6842F001021A60002016
:1064F8007047012070470020704700BF000001402E
:106508000700010030B50368394A904214BF4FF0C4
:10651800000E4FF0010EB0F1804F14BF72464EF0DE
:106528000102AAB9334CA04214BF00240124324D01
:10653800A8420DD064B904F1804404F58234A04225
:1065480014BF0024012405F50065A84200D01CB141
:1065580023F070034C68234312BB264A904214BFB1
:1065680000220122244CA0421AD0CAB902F180426A
:1065780002F58232904214BF0022012204F5006421
:10658800A0420DD062B91D4A904214BF00220122D8
:1065980004F59A34A04203D012B9194A904204D1A2
:1065A80023F4407CCB6843EA0C0323F080034A6958
:1065B800134303608A68C2620A688262114A904281
:1065C80014BF73464EF0010363B90C4B984214BFD5
:1065D8000023012302F57052904203D013B9084BEF
:1065E800984201D10B6903630123436130BD00BFA9
:1065F8000000014000080040000400400044014041
:10660800004801400004014060B310B5044690F80A
:106618003D3013B3022384F83D30214651F8040B72
:10662800FFF770FF012384F8483084F83E3084F87F
:106638003F3084F8403084F8413084F8423084F8A0
:10664800433084F8443084F8453084F8463084F880
:10665800473084F83D30002010BD80F83C30FCF70E
:1066680097F8D7E70120704710B4846824F47F4C6A
:1066780042EA03220A4342EA0C02826010BC7047D5
:1066880090F83C30012B00F08F8010B504460123B0
:1066980080F83C30022380F83D3002689068434B14
:1066A800034093600B68702B55D031D8502B6CD0B9
:1066B8000CD9602B2AD1CA6849682068FFF7C0FE48
:1066C80060212068FFF7D0FE002035E0402B0AD17A
:1066D800CA6849682068FFF7A1FE40212068FFF7D3
:1066E800C3FE002028E05BD8202B07D003D9302B2D
:1066F80004D0012020E00BB1102B05D119462068E9
:10670800FFF7B2FE002017E0012015E0012013E09A
:10671800B3F5005F2CD00BD9254A9342EED012D99D
:10672800244A9342EAD010329342E7D0012003E092
:10673800B3F5805F36D10020012384F83D30002373
:1067480084F83C3010BDB3F5801FD7D0B3F1101FCB
:10675800D4D00120F0E7CB684A6889682068FFF741
:1067680083FF2268936843F0770393600020E3E790
:10677800CB684A6889682068FFF776FF22689368C3
:1067880043F4804393600020D6E7CA6849682068CC
:10679800FFF744FE50212068FFF766FE0020CBE794
:1067A8000120C9E70120C7E7022070478800CEFF13
:1067B800200010003000100090F83C30012B45D02C
:1067C80070B4012380F83C30022380F83D30036820
:1067D8005A689C681E4E1F4DAB4218BFB34203D186
:1067E80022F470024D682A4322F070020D682A4391
:1067F8005A600368164AB3F1804F18BF934217D006
:10680800A2F57C42934213D002F5806293420FD0E6
:1068180002F5806293420BD002F57842934207D08A
:10682800A2F56C42934203D002F59432934204D10C
:1068380024F080048A6814439C60012380F83D306A
:10684800002380F83C30184670BC7047022070471F
:106858000000014000040140026852E8003F23F0B4
:10686800C00342E800310029F6D1026802F10803AA
:1068780053E8003F23F40003083242E800310029BE
:10688800F3D12023C0F8843070470000026852E832
:10689800003F23F4907342E800310029F6D10268E2
:1068A80002F1080353E8001F0D4B0B40083242E881
:1068B80000310029F3D1C36E012B06D02023C0F884
:1068C80088300023C36603677047026852E8003FB8
:1068D80023F0100342E800310029F6D1EEE700BFAB
:1068E800FEFFFFEF1346D0F88420202A4AD110B5C6
:1068F8000446002B18BF002946D090F88020012AB2
:1069080044D0012280F880200165A0F85430A0F816
:1069180056300022C0F88C202122C0F88420826FD3
:10692800E2B11B49D163826F1A491164826F1A4917
:10693800D164826F0021116502682832016D806F71
:10694800FCF746FE50B11023C4F88C30002384F8BD
:1069580080302023C4F88430012012E023684022CC
:106968001A62002384F88030226802F1080353E891
:10697800003F43F08003083242E800310029F3D198
:10698800002010BD022070470120FAE70220F8E736
:10699800556A0008C16A0008CF6A000838B504467D
:1069A800D0F88420D0F8885003689B6813F0800FD3
:1069B80001D0212A08D023689B6813F0400F42D0E9
:1069C800222D20D000203FE0226802F1080353E87E
:1069D800003F23F08003083242E800310029F3D158
:1069E800A06F10B1FCF740FF18B92046FFF734FF3D
:1069F800E1E7A06FFDF7ACFD2028F6D11023C4F81D
:106A08008C30032020E0226802F1080353E8003F9D
:106A180023F04003083242E800310029F3D1E06F47
:106A280010B1FCF721FF20B92046FFF72FFF002007
:106A38000AE0E06FFDF78CFD2028F5D11023C4F89B
:106A48008C30032000E0002038BD704708B50346AD
:106A5800806BDB69B3F5807F18D00023A0F856302F
:106A6800026802F1080353E8003F23F0800308326C
:106A780042E800310029F3D1026852E8003F43F0B0
:106A8800400342E800310029F6D108BDFFF7DDFFD9
:106A9800FBE708B5026852E8003F23F0400342E8EC
:106AA80000310029F6D12023C0F884300023436741
:106AB800FFF7CBFF08BD704708B5806BFFF7FBFFFA
:106AC80008BD7047704738B5846BD4F88420D4F873
:106AD800885023689B6813F0800F01D0212A10D0BA
:106AE80023689B6813F0400F01D0222D10D0D4F8F2
:106AF8008C3043F01003C4F88C302046FFF7E2FFD7
:106B080038BD0023A4F856302046FFF7A5FEE7E776
:106B18000023A4F85E302046FFF7B8FEE7E708B583
:106B2800806B0023A0F85E30A0F85630FFF7CAFF4C
:106B380008BD704770B504460168CB6908688D6860
:106B480040F60F021A4008D113F0200F05D010F0BC
:106B5800200F34D115F0805F31D12AB1894A2A40FB
:106B680033D1894E304230D1E26E012A00F0C38021
:106B780013F4801F03D015F4800F40F0928113F0B6
:106B8800800F07D010F0800F40F0928115F4000FAD
:106B980040F08E8113F0400F03D010F0400F40F00A
:106BA8008E8113F4000F03D010F0804F40F08B81DA
:106BB80013F0807F02D00028C0F2898170BD236F56
:106BC800002BFBD020469847F8E713F0010F09D0B7
:106BD80010F4807F06D001260E62D4F88C10314361
:106BE800C4F88C1013F0020F0BD015F0010F08D069
:106BF800216802260E62D4F88C1041F00401C4F812
:106C08008C1013F0040F0BD015F0010F08D0216879
:106C180004260E62D4F88C1041F00201C4F88C10DE
:106C280013F0080F0BD010F0200F00D13AB12268F2
:106C380008211162D4F88C200A43C4F88C2013F47C
:106C4800006F0CD010F0806F09D022684FF40061FB
:106C58001162D4F88C2042F02002C4F88C20D4F8B9
:106C68008C20002AAAD013F0200F09D010F0200F92
:106C780002D115F0805F03D0236F0BB120469847EF
:106C8800D4F88C2023689B6813F0400F02D112F0CF
:106C9800280F29D02046FFF7F9FD23689B6813F0D9
:106CA800400F1DD0226802F1080353E8003F23F08B
:106CB8004003083242E800310029F3D1E36F5BB1A9
:106CC800324A1A65E06FFCF76FFF00283FF476AF91
:106CD800E06F036D984771E72046FFF7F3FE6DE715
:106CE8002046FFF7EFFE69E72046FFF7EBFE00239B
:106CF800C4F88C3062E713F0100F3FF439AF10F08E
:106D0800100F3FF435AF10230B6223689B6813F014
:106D1800400F00F08E80E26F13681D481D498B42BA
:106D280018BF834238D018318B4235D018318B4286
:106D380032D018318B422FD018318B422CD01831D9
:106D48008B4229D018318B4226D001F556718B42DF
:106D580022D018318B421FD018318B421CD01831E9
:106D68008B4219D018318B4216D018318B4213D070
:106D780018318B4210D018318B420DD05B689BB212
:106D88000CE000BF0100001020010004276B000880
:106D980010000240280002405B689BB2002B3FF4C1
:106DA8000DAFB4F85C1099427FF608AFA4F85E30D6
:106DB800D369B3F5807F31D0226852E8003F23F4CD
:106DC800807342E800310029F6D1226802F10803F5
:106DD80053E8003F23F00103083242E8003100295C
:106DE800F3D1226802F1080353E8003F23F040037F
:106DF800083242E800310029F3D12023C4F8883052
:106E08000023E366226852E8003F23F0100342E8BB
:106E180000310029F6D1E06FFCF726FDB4F85C10CC
:106E2800B4F85E309BB2C91A89B22046FFF781FEDA
:106E3800C4E6B4F85C10B4F85E309BB2C91A89B2E3
:106E4800B4F85E309BB2002B3FF4B8AE00293FF493
:106E5800B5AE226852E8003F23F4907342E8003050
:106E68000028F6D1226802F1080353E8000F1A4BF4
:106E78000340083242E800300028F3D12023C4F848
:106E880088300023E3662367226852E8003F23F036
:106E9800100342E800300028F6D12046FFF749FEEB
:106EA8008CE64FF480130B62204601F0E3F885E688
:106EB800636F002B3FF482AE204698477EE620465B
:106EC800FFF7E7FD7AE6204601F0D6F876E6204699
:106ED80001F0D1F872E600BFFEFFFFEF08B5B0F889
:106EE8006030D0F88820222A05D00268936943F0E0
:106EF8000803936108BD0268516ADBB2826D0B40DA
:106F08001370836D01338365B0F85E309BB2013B2B
:106F18009BB2A0F85E30B0F85E309BB2002BE9D18E
:106F2800026852E8003F23F4907342E800310029D8
:106F3800F6D1026802F1080353E8003F23F0010389
:106F4800083242E800310029F3D12023C0F8883004
:106F580000230367C36E012B16D10023C3660268A2
:106F680052E8003F23F0100342E800310029F6D12F
:106F78000368DA6912F0100F01D010221A62B0F813
:106F88005C10FFF7D6FDB5E7FAF734FFB2E708B5AE
:106F9800B0F86020D0F88830222B05D002689369B9
:106FA80043F00803936108BD03685B6A816D134071
:106FB8000B80836D02338365B0F85E309BB2013B72
:106FC8009BB2A0F85E30B0F85E309BB2002BEAD1DD
:106FD800026852E8003F23F4907342E80031002928
:106FE800F6D1026802F1080353E8003F23F00103D9
:106FF800083242E800310029F3D12023C0F8883054
:1070080000230367C36E012B16D10023C3660268F1
:1070180052E8003F23F0100342E800310029F6D17E
:107028000368DA6912F0100F01D010221A62B0F862
:107038005C10FFF77EFDB6E7FAF7DCFEB3E7000069
:107048002DE9F843B0F860600368DD69D3F8009073
:10705800D3F80880D0F88820222A05D09A6942F00F
:1070680008029A61BDE8F8830446B0F8687008E041
:10707800D4F88C30002B4CD1B4F85E309BB2002B86
:107088004ED0002F00F0858015F0200F00F0818091
:107098002368596AF3B2A26D0B401370A36D0133D4
:1070A800A365B4F85E309BB2013B9BB2A4F85E3096
:1070B8002368DD6915F0070FDED015F0010F09D040
:1070C80019F4807F06D001221A62D4F88C30134359
:1070D800C4F88C3015F0020F0BD018F0010F08D04F
:1070E800236802221A62D4F88C3043F00403C4F8EF
:1070F8008C3015F0040FBBD018F0010FB8D02368FE
:1071080004221A62D4F88C3043F00203C4F88C309D
:10711800AEE72046FFF7D6FC0023C4F88C30ABE777
:10712800226852E8003F23F4807342E800310029C6
:10713800F6D1226802F1080353E8001F264B0B40E2
:10714800083242E800310029F3D12023C4F88830FE
:1071580000232367E36E012B03D02046FAF74AFE8B
:107168008FE70023E366226852E8003F23F010030C
:1071780042E800310029F6D12368DA6912F0100FCD
:1071880001D010221A62B4F85C102046FFF7D1FC37
:1071980077E7B4F85E309BB2002B3FF463AFB4F8E6
:1071A80068209A427FF65EAF226802F1080353E82E
:1071B800003F23F08053083242E800310029F3D120
:1071C800064B2367226852E8003F43F0200342E859
:1071D80000310029F6D145E7FEFFFFEFE56E000814
:1071E8002DE9F843B0F860600368DD69D3F80090D2
:1071F800D3F80880D0F88820222A05D09A6942F06E
:1072080008029A61BDE8F8830446B0F8687008E09F
:10721800D4F88C30002B4AD1B4F85E309BB2002BE6
:107228004CD0002F00F0838015F0200F7FD023680A
:107238005B6AA26D33401380A36D0233A365B4F873
:107248005E309BB2013B9BB2A4F85E302368DD69D7
:1072580015F0070FE0D015F0010F09D019F4807F61
:1072680006D001221A62D4F88C301343C4F88C304B
:1072780015F0020F0BD018F0010F08D02368022276
:107288001A62D4F88C3043F00403C4F88C3015F03B
:10729800040FBDD018F0010FBAD0236804221A6277
:1072A800D4F88C3043F00203C4F88C30B0E72046A1
:1072B800FFF708FC0023C4F88C30ADE7226852E8D9
:1072C800003F23F4807342E800310029F6D1226898
:1072D80002F1080353E8001F264B0B40083242E82E
:1072E80000310029F3D12023C4F888300023236714
:1072F800E36E012B03D02046FAF77CFD91E70023CB
:10730800E366226852E8003F23F0100342E80031A8
:107318000029F6D12368DA6912F0100F01D0102283
:107328001A62B4F85C102046FFF703FC79E7B4F85A
:107338005E309BB2002B3FF465AFB4F868209A42E8
:107348007FF660AF226802F1080353E8003F23F09C
:107358008053083242E800310029F3D1064B2367F5
:10736800226852E8003F43F0200342E80031002938
:10737800F6D147E7FEFFFFEF976F000808B5806B6F
:10738800C36E012B02D0FFF79CFB08BDB0F85C1060
:107398004908FFF7CEFBF8E708B50346806BDB69C1
:1073A800B3F5807F29D00023A0F85E30026852E848
:1073B800003F23F4807342E800310029F6D10268C7
:1073C80002F1080353E8003F23F00103083242E8C2
:1073D80000310029F3D1026802F1080353E8003FA5
:1073E80023F04003083242E800310029F3D120237A
:1073F800C0F88830C36E012B05D0C36E012B0CD0AA
:10740800FAF7F8FC08BD026852E8003F23F01003C1
:1074180042E800310029F6D1EFE7B0F85C10FFF739
:1074280088FBEFE770B586B0044601688368026997
:10743800134342691343C26913430868884A0240E8
:1074480013430B602268536823F44053E1680B43ED
:107458005360A1692268834B9A4201D0236A194379
:107468009068814B03400B4393602268D36A23F0F2
:107478000F03616A0B43D36222687C4B9A4221D086
:107488007B4B9A4200F08C807A4B9A4200F0A280A3
:10749800794B9A4200F0B580784B9A4200F0C88048
:1074A800774B9A4200F0F480764B9A4200F01981AB
:1074B800754B9A4200F02C816A4B9A4200F03F814A
:1074C800802333E0714B5B6D03F03803282B65D8BC
:1074D800DFE813F0290064006400640064006400BD
:1074E800640064004D01640064006400640064008A
:1074F800640064002B00640064006400640064009D
:10750800640064005E006400640064006400640059
:107518006400640060006400640064006400640047
:10752800640064006200012300E008234D498A4298
:1075380000F02F81E069B0F5004F00F0AF81202BFB
:1075480000F20782202B00F25182DFE813F01E02BE
:1075580024024F024F0227024F024F024F022C0211
:107568004F024F024F024F024F024F024F023102A9
:107578004F024F024F024F024F024F024F024F027B
:107588004F024F024F024F024F024F024F023D027D
:107598001023CBE72023C9E74023C7E78023C5E7AB
:1075A8003A4B5B6D03F00703052B11D8DFE813F0A6
:1075B8000600E10008000A000C000E000023B5E7F1
:1075C8000823B3E71023B1E72023AFE74023ADE753
:1075D8008023ABE72D4B5B6D03F00703052B0ED81B
:1075E800DFE803F003C90507090B00239EE708231A
:1075F8009CE710239AE7202398E7402396E7802307
:1076080094E7224B5B6D03F00703052B0ED8DFE8E8
:1076180003F003B40507090B002387E7082385E770
:10762800102383E7202381E740237FE780237DE73A
:10763800164B5B6D03F00703052B0ED8DFE803F04C
:10764800039F0507090B002370E708236EE7102343
:107658006CE720236AE7402368E7802366E700BFDA
:10766800F369FFCF000C0058FFF4FF110010014030
:107678000044004000480040004C004000500040DA
:107688000014014000780040007C0040004402588B
:107698007D4B5B6D03F03803282B20D8DFE803F01F
:1076A800151F1F1F1F1F1F1F711F1F1F1F1F1F1F9A
:1076B800171F1F1F1F1F1F1F191F1F1F1F1F1F1FE0
:1076C8001B1F1F1F1F1F1F1F1D0001232EE708233D
:1076D8002CE710232AE7202328E7402326E78023E6
:1076E80024E7694B5B6D03F00703052B0ED8DFE831
:1076F80003F0034A0507090B002317E7082315E7DA
:10770800102313E7202311E740230FE780230DE719
:107718005D4B5B6D03F00703052B0ED8DFE803F024
:1077280003350507090B002300E70823FEE61023AD
:10773800FCE62023FAE64023F8E68023F6E603F584
:107748000E339B6D03F00703052B0ED8DFE803F01B
:10775800031F0507090B0223E8E60823E6E61023C2
:10776800E4E62023E2E64023E0E68023DEE6042385
:10777800DCE60423DAE60423D8E60423D6E6042369
:10778800D4E60423D2E60423D0E60423CEE6042379
:10779800CCE6202B27D8022BC0F01A81023B1E2BE7
:1077A80000F21881DFE813F05000160156001601A8
:1077B800160116015B0016011601160116011601C5
:1077C80016011601600016011601160116011601B0
:1077D80016011601160116011601160116011601E9
:1077E800160116016C00402B2CD14FF40040626A40
:1077F800264B33F81220B0FBF2F3656805EB450120
:10780800994200F2E980B3EB053F00F2E7800026D9
:1078180033463146F9F7C8FC090241EA1061000213
:107828006B08C0182A46334641F10001F9F7BCFC41
:10783800A0F54072164B9A4200F2D2802368D860B5
:107848003046D4E00120D2E0FEF7A2FB0028CED1DA
:107858000020CCE003A8FEF7ADFB0498F6E76846E5
:10786800FEF7C2FC0198F1E7074B1B6813F0200FE5
:1078780008D0054B1B68C3F3C1030648D840E5E7A9
:107888000548B4E70348B2E70044025810980008D6
:10789800FFFC0F000090D00300093D00202B15D8F5
:1078A800202B00F29F80DFE803F031379D9D3A9D41
:1078B8009D9D3F9D9D9D9D9D9D9D449D9D9D9D9DA7
:1078C8009D9D9D9D9D9D9D9D9D9D5000402B1BD1E7
:1078D800626A4D4B33F81230B0FBF3F0626853081C
:1078E80003EB4000B0FBF2F0A0F110024FF6EF738B
:1078F8009A4279D883B223F00F03C0F342001843A9
:107908002368D860002072E0012070E0FDF72EFDAA
:107918000028DDD100206AE0FDF73AFDF8E703A86A
:10792800FEF748FB0498F3E76846FEF75DFC01980C
:10793800EEE7364B1B6813F0200F08D0334B1B685B
:10794800C3F3C1033248D840E2E73248C0E73048C1
:10795800BEE7402B17D14FF40040626A2A4B33F838
:107968001230B0FBF3F0636800EB5300B0FBF3F0A8
:10797800A0F110024FF6EF739A4242D8236880B202
:10798800D860002033E0012031E0FDF7EFFC00284B
:10799800E3D100202BE0FDF7FBFCF8E703A8FEF796
:1079A80009FB0498F3E76846FEF71EFC0198EEE72A
:1079B800164B1B6813F0200F08D0144B1B68C3F339
:1079C800C1031348D840E2E71248C6E71048C4E7A5
:1079D80001200CE001200AE0012008E0012006E077
:1079E800012004E0012002E0012000E00120012341
:1079F800A4F86A30A4F8683000232367636706B0E8
:107A080070BD0120F3E700BF109800080044025839
:107A18000090D00300093D00836A13F0010F06D0DF
:107A28000268536823F40033C16A0B435360836AC6
:107A380013F0020F06D00268536823F48033016BF9
:107A48000B435360836A13F0040F06D0026853682F
:107A580023F48023416B0B435360836A13F0080FB0
:107A680006D00268536823F40043816B0B435360CC
:107A7800836A13F0100F06D00268936823F48053CA
:107A8800C16B0B439360836A13F0200F06D0026822
:107A9800936823F40053016C0B439360836A13F0DB
:107AA800400F0AD00268536823F48013416C0B43DB
:107AB8005360436CB3F5801F0BD0836A13F0800FBB
:107AC80006D00268536823F40023C16C0B4353604B
:107AD80070470268536823F4C003816C0B435360FA
:107AE800EBE72DE9F84305460F4616469946DDF8BB
:107AF80020802C68E46937EA04030CBF4FF0010CBE
:107B08004FF0000CB44557D1B8F1FF3FF1D0FBF767
:107B180005F8A0EB090040452FD8B8F1000F2CD08C
:107B28002B681A6812F0040FE3D0DA6912F4006FB8
:107B3800DFD04FF400621A622A6852E8003F23F44B
:107B4800D07342E800310029F6D12A6802F108030F
:107B580053E8003F23F00103083242E800310029CE
:107B6800F3D12023C5F88430C5F88830C5F88C30A7
:107B7800002385F8803003201FE02A6852E8003F80
:107B880023F4D07342E800310029F6D12A6802F1C3
:107B9800080353E8003F23F00103083242E80031AC
:107BA8000029F3D12023C5F88430C5F88830002394
:107BB80085F88030032000E00020BDE8F8832DE937
:107BC800F04182B01E46D0F88430202B58D10446AC
:107BD8000D469046002A18BF002955D090F88030ED
:107BE800012B53D0012380F880300023C0F88C305B
:107BF8002123C0F88430FAF791FF0746A4F854808F
:107C0800A4F85680A368B3F5805F05D04FF000084C
:107C1800002384F8803012E0236913B14FF0000884
:107C2800F6E7A8460025F3E715F8012B23689A62C2
:107C3800B4F8562092B2013A92B2A4F85620B4F899
:107C480056309BB283B100963B46002280212046E5
:107C5800FFF747FFE0B9002DE6D138F8023B22686C
:107C6800C3F308039362E3E700963B4600224021F2
:107C78002046FFF736FF68B92023C4F8843000E0B7
:107C8800022002B0BDE8F0810120FAE70220F8E7FF
:107C98000320F6E70320F4E730B583B00446002359
:107CA800C0F88C30FAF73AFF05462268126812F0DD
:107CB800080F0FD123681B6813F0040F18D1202375
:107CC800C4F88430C4F888300020E06684F8800066
:107CD80003B030BD6FF07E430093034600224FF49B
:107CE80000112046FFF7FDFE0028E3D00320EFE750
:107CF8006FF07E4300932B4600224FF4800120460C
:107D0800FFF7EFFE0028DAD00320E1E778B310B5DB
:107D18000446D0F884300BB32423C4F88430226896
:107D2800136823F0010313602046FFF77BFB01284B
:107D380013D0A36ABBB92268536823F490435360F5
:107D48002268936823F02A0393602268136843F03B
:107D5800010313602046FFF79FFF10BD80F88030B5
:107D6800FAF798FDD8E72046FFF756FEE3E701202B
:107D78007047000010B48165A0F85C20A0F85E2070
:107D8800002303678368B3F5805F06D0A3B903694E
:107D980073B9FF23A0F8603014E0036923B940F2F7
:107DA800FF13A0F860300DE0FF23A0F8603009E071
:107DB8007F23A0F8603005E0B3F1805F30D0002366
:107DC800A0F860300023C0F88C302223C0F8883037
:107DD800016801F1080353E8003F43F0010308314B
:107DE80041E80034002CF3D1436EB3F1005F21D099
:107DF8008368B3F5805F48D02C4B0367002380F875
:107E080080300369002B46D0026852E8003F43F4F3
:107E1800907342E800310029F6D1002010BC704769
:107E280003691BB97F23A0F86030CBE73F23A0F894
:107E38006030C7E7B0F868309342D9D88368B3F5A3
:107E4800805F1CD01A4B0367002380F880300369D9
:107E580043B1026852E8003F43F4807342E80031BE
:107E68000029F6D1026802F1080353E8003F43F005
:107E78008053083242E800310029F3D1CDE7036985
:107E8800002BDFD10B4B0367DEE70369002BB3D16F
:107E9800094B0367B2E7026852E8003F43F020034A
:107EA80042E800310029F6D1B7E700BFE56E0008C7
:107EB80049700008E9710008976F000838B5D0F8D4
:107EC8008830202B20D1002A18BF00291ED090F816
:107ED8008030012B1CD0012380F880300023C3663A
:107EE80003680C4CA3420CD05B6813F4000F08D055
:107EF800046854E8003F43F0806344E80035002DEF
:107F0800F6D1FFF737FF00E0022038BD0120FCE77B
:107F18000220FAE7000C005810B5044613468165A4
:107F2800A0F85C200022C0F88C202222C0F888200B
:107F3800C26F8AB12249D163C26F22491164C26FEC
:107F48002149D164C26F002111650168826D243115
:107F5800C06FFBF73DFB38BB002384F880302369F2
:107F680043B1226852E8003F43F4807342E800318D
:107F78000029F6D1226802F1080353E8003F43F0D4
:107F88000103083242E800310029F3D1226802F1E6
:107F9800080353E8003F43F04003083242E8003149
:107FA8000029F3D1002010BD1023C4F88C30002321
:107FB80084F880302023C4F888300120F3E700BF1C
:107FC800A173000885730008CF6A000838B5D0F897
:107FD8008830202B20D1002A18BF00291ED090F805
:107FE8008030012B1CD0012380F880300023C36629
:107FF80003680C4CA3420CD05B6813F4000F08D044
:10800800046854E8003F43F0806344E80035002DDD
:10801800F6D1FFF781FF00E0022038BD0120FCE720
:108028000220FAE7000C0058436E2BB90123A0F890
:108038006A30A0F86830704730B403689A68C2F3B1
:1080480042629968490F094D6B5C1B01084C615CE1
:1080580093FBF1F3A0F86A30AB5C1B01A25C93FBC5
:10806800F2F3A0F8683030BC704700BF30980008C1
:108078002898000870477047704790F88030012BA7
:1080880018D0012380F880302423C0F88430036896
:108098001A68196821F00101196022F000520023C2
:1080A800436601680A602022C0F8842080F8803086
:1080B800184670470220704738B590F88030012B79
:1080C8001DD00446012380F880302423C0F8843072
:1080D80003681D681A6822F001021A600268936832
:1080E80023F0604319439160FFF79EFF23681D60EA
:1080F8002023C4F88430002084F8800038BD022092
:10810800FCE738B590F88030012B1DD004460123D8
:1081180080F880302423C0F8843003681D681A680A
:1081280022F001021A600268936823F06063194321
:108138009160FFF779FF23681D602023C4F884301D
:10814800002084F8800038BD0220FCE7014B186845
:10815800704700BF2000002470B50D4E0D4D761BF2
:10816800B61006D0002455F8043B01349847A642BF
:10817800F9D1094E094D761B01F02CFBB61006D03B
:10818800002455F8043B01349847A642F9D170BD44
:10819800789800087898000880980008789800086F
:1081A800830730B548D0541E002A3FD0CAB20346D0
:1081B80001E0013C3AD303F8012B9D07F9D1032CC8
:1081C8002DD9CDB245EA05250F2C45EA054536D906
:1081D800A4F1100222F00F0C03F1200EE6444FEA3E
:1081E800121C03F1100242E9045542E9025510320B
:1081F8007245F8D10CF1010214F00C0F03EB0212D6
:1082080004F00F0C13D0ACF1040323F00303043380
:10821800134442F8045B9342FBD10CF003042CB1E5
:10822800CAB21C4403F8012B9C42FBD130BD644602
:108238001346002CF4D1F9E703461446BFE71A4663
:10824800A446E0E72DE9F043694CD4F8008083B0F8
:1082580004460E4617461D46B8F1000F03D0D8F85D
:108268003830002B77D0022F05D0012F00F2AC80D8
:10827800002DC0F2A980636EDA0752D52146404628
:1082880000F058F9216B41B104F14003994202D042
:10829800404600F07BFA00232363B4F90CC00023A6
:1082A8001CF0800FA361636064D12CF44A6C2CF03D
:1082B800030C022FA4F80CC06AD001AB6A46214611
:1082C800404600F095FBA3891843A081002D2FD0CC
:1082D800002E2ED0D8F83830002B38D0009B2660DE
:1082E800AB42B4F90C301CBF43F40063A381012FE7
:1082F80004BF43F00103A3819AB213F00803C4E951
:1083080004652CD0D1075DD56D42A561656E00234B
:1083180015F00105A36027D00025284603B0BDE865
:10832800F083A3899B05A9D4A06D00F05DFBA5E7A8
:10833800009D284600F08CFB0646002847D0A389FC
:1083480043F08003A381D8F83830002BC6D14046CB
:1083580000F024F9C2E7404600F020F983E7A36063
:10836800656E15F00105D7D1930524D5284603B0CD
:10837800BDE8F0832169404600F008FAB4F90CC062
:108388002CF44A6C2CF0030C022FA4F80CC094D1E6
:108398000025002204F14303A2600122C4E904324B
:1083A8002360636E4CF0020CD807A4F80CC0DDD42F
:1083B8001CF4007FDAD1A06D00F018FB284603B04A
:1083C800BDE8F083A560CBE74FF0FF35CEE7DDF8D9
:1083D8000090A94504D0484600F03AFB064620B96B
:1083E800B4F90CC04FF0FF35D3E74D46A7E700BFFF
:1083F80020000024024B13B1024800F005B8704772
:1084080000000000C9860008002301461A461846E5
:1084180000F050BEB1F90C20F8B50C46110707461C
:1084280042D4636842F40062002BA28159DDA56A38
:10843800002D54D000233E683B6093B212F4805262
:1084480053D1E16901233846A847421C63D0A38968
:10845800A56A5B0705D56368C01A236B0BB1E36B8C
:10846800C01AE169024600233846A847411C3ED19C
:108478003B68002B3BD01D2B01D0162B52D1A38972
:108488002269226023F4006300216160A381216BCB
:108498003E6021B304F14003994202D0384600F00F
:1084A80075F900202063F8BD2669C6B193B2256826
:1084B80026609A070CBF63690023AD1BA3600CE01C
:1084C800D4F824C0E1692B4632463846E047B0F17B
:1084D800000CA5EB0C05664416DD002DF0DC002031
:1084E800F8BDE36B002BA2DCF9E7206DB1E7B4F926
:1084F8000C302269226023F40063A3810022DB048C
:108508006260C4D52065C2E7A38943F040034FF0F9
:10851800FF30A381F8BD3B68002B98D01D2B06D0F7
:10852800162B04D0A38943F04003A381F8BD3E6015
:10853800D5E700BF38B50C46054608B1836BA3B133
:10854800B4F90C00B8B1636EDB0701D4810515D509
:1085580028462146FFF75EFF636EDA07054602D418
:10856800A3899B050ED5284638BD00F017F8B4F945
:108578000C000028E7D10546284638BDA06D00F05C
:1085880033FAE5E7A06D00F031FA284638BD00BFA0
:10859800014900F001BA00BF6D9100082DE9F047CC
:1085A8008246394800F020FADAF83840002C66D1C3
:1085B800DAF80450354ACAF83C200323CAE9B8431C
:1085C800DFF8CC90DFF8CC80334F344E04230AF523
:1085D8003B72CAF8E8222146C5E90243C5E90044CE
:1085E800C5E904446C660822AC6105F15C00FFF73C
:1085F800D7FDC5E90759C5E90987EE6205F15800B5
:1086080000F0EEF9DAF80850254BEB602146C5E991
:108618000044C5E904446C66AC60AC61082205F10D
:108628005C00FFF7BDFDC5E90759C5E90987EE629A
:1086380005F1580000F0D4F9DAF80C50194BEB604A
:108648002146C5E90044C5E904446C66AC60AC61E8
:10865800082205F15C00FFF7A3FD05F15800C5E904
:108668000759C5E90A76C5F8248000F0B9F901234D
:10867800CAF838300448BDE8F04700F0B7B9BDE89B
:10868800F047014800F0B2B92C440024998500084D
:108698000590000829900008699000088990000852
:1086A8000900010012000200014800F09DB900BF56
:1086B80028440024014800F099B900BF2844002448
:1086C80038B5084B084D5B1B9C1007D0043B1D4474
:1086D800013C55F804399847002CF9D1BDE83840D9
:1086E80001F07EB88498000880980008F8B5244FF7
:1086F8000C46064600F064FCBA685568C4F57E630B
:108708000F3325F003052B4423F47F6323F00F0375
:10871800A3F58054B4F5805F07DB0021304600F0F4
:108728005BFCBB682B44984204D0304600F04EFCFA
:108738000020F8BD6142304600F04EFC01300DD0FB
:10874800104ABB682D1B45F001055D601368304673
:108758001B1B136000F03AFC0120F8BD00213046D5
:1087680000F03AFCBA68831A0F2BDEDD43F00103F0
:108778005360054B03491B68C01A0860D5E700BF62
:1087880054040024304400245C080024002961D0EB
:10879800F8B50C46064600F013FC54F8042C7B4F41
:1087A800A4F1080522F0010105EB010CB868DCF81A
:1087B8000430604523F0030300F08B80D207CCF827
:1087C800043032D454F8082CAD1A1144AA6807F1C1
:1087D800080082426AD00CEB0304D4F804E0EC6889
:1087E800D4601EF0010FA26000F0978041F00103F1
:1087F8006B60CCF80010B1F5007F35D27A68CB08F1
:1088080048090121013381401143796007EBC30214
:1088180057F83310083AC5E9021247F83350CD60CB
:108828003046BDE8F84000F0D1BB0CEB03025268BB
:10883800D00710D4194407F10800DCF80830834247
:1088480073D0DCF80C20DA60936041F001036B60B0
:108858006950D0E7704741F00103B1F5007F44F853
:10886800043CCCF80010C9D3B1F5206F4FEA51236E
:1088780048D28B0903F1390003F13802C300F81814
:10888800FB580838984259D05A6822F003028A42A5
:1088980002D99B689842F7D1D868C5E9023085604B
:1088A800DD603046BDE8F84000F090BB0CEB0302F9
:1088B8005268D20763D40B44DCE90212CA609160A3
:1088C80043F001026A603046EB50BDE8F84000F022
:1088D8007DBB0B44D10707D454F8082CAD1A1344B8
:1088E800D5E90212CA60916043F001026A60284A21
:1088F800BD6012689A4293D8264B30461968FFF734
:10890800F5FE8DE7142B0AD9542B1FD80B0B03F156
:108918006F0003F16E02C300B1E719448DE703F15C
:108928005C0003F15B02C300A9E741F00103C7E95A
:108938000455C5E902006B60695071E779689210C7
:10894800012404FA02F20A437A60A6E7B3F5AA7F83
:1089580006D8CB0B03F1780003F17702C3008EE74A
:1089680040F25452934206D88B0C03F17D0003F178
:108978007C02C30083E74FF47E737E227FE741F0D9
:1089880001036B60CCF800104AE700BF54040024D0
:1089980060080024604400242DE9F843074688460F
:1089A80000F538764FF00009D6E90154013D11D49D
:1089B800A389012B05F1FF3508D9B4F90E3001332D
:1089C800214603D03846C04749EA00096B1C04F128
:1089D8006804EDD13668002EE6D14846BDE8F88334
:1089E800704700BF704700BF704700BF704700BFA7
:1089F80070B50C46B1F90E10002996B015461E4602
:108A080014DB6A4600F014FC00280FDB019A02F41C
:108A18007042A2F50052B2FA82F24FF48063520912
:108A28004FF4006032602B6016B070BDB4F90C10C2
:108A3800002311F08000336004D0402218462A60D9
:108A480016B070BD4FF480632B6016B070BD00BFC8
:108A5800024B0146186800F003B800BF200000244C
:108A68002DE9F04F01F10B06162E83B0044624D8E9
:108A7800102900F2BA8000F0A3FA1026182202206A
:108A8800B54F3A44A2F1080153688B4200F0BA800E
:108A98005A68D96822F003021A449D68E9608D601B
:108AA800516841F001012046516003F1080500F0CA
:108AB8008DFA284603B0BDE8F08F36F0070600F1BE
:108AC8009480B14200F2918000F07AFAB6F5FC7F0A
:108AD800C0F09A81730A00F08F80042B00F26F8136
:108AE800B30903F1390003F1380CC3009A4F3B4432
:108AF800A3F108055B689D4206D10CE0002980F2CD
:108B08002781DB689D4206D05A6822F00302911B38
:108B18000F29F3DD60463D69DFF840C265457CD02A
:108B28006A6822F00302931B0F2B00F37B81002B52
:108B3800C7E904CC80F26C81B2F5007F80F01A811D
:108B4800D308796801334FEA521E012202FA0EF265
:108B58000A4357F833E0C5F808E007EBC3010839C2
:108B6800E9607A6047F83350CEF80C508310012141
:108B78009940914257D8114206D120F0030049008C
:108B8800114200F10400FAD007EBC0094D468646B1
:108B9800D5F80C80454508D11DE1002B80F22481D1
:108BA800D8F80C80454500F01681D8F8042022F04A
:108BB8000302931B0F2BF0DD2046D8E9025408EB83
:108BC800060146F00106C8F80460EC60A56043F0B1
:108BD8000104C7E90411C1E902CC4C6048F802302D
:108BE80000F0F4F908F1080502E00C2323600025E1
:108BF800284603B0BDE8F08F4FF4007340204FF0D3
:108C08003F0C73E7D3689A4208BF02307FF440AF45
:108C18003D69DFF848C1654582D17A688310012132
:108C280099409142A7D9BD686B6823F003094E4566
:108C380003D8A9EB06030F2B7ADCDFF824B1494BE4
:108C4800DBF800201B680132334405EB090A00F009
:108C5800338103F580530F3323F47F6828F00F081E
:108C68004146204600F0B8F9411C024600F0F38066
:108C7800824500F2EE803C4B196841441960084671
:108C880000F04E81DBF80010019301311BBFA2EB0D
:108C98000A0A5044CBF80020186012F0070B00F0C5
:108CA8001781CBF108010A44CBF580519044083173
:108CB800A1EB0801C1F30B0A51462046009200F0CF
:108CC8008BF9421CDDE9002300F04F81801A00EB8C
:108CD8000A081968BA6048F001005144BD42506062
:108CE800196000F02981B9F10F0F40F227816868F7
:108CF800A9F10C0C2CF0070C00F0010040EA0C0064
:108D080068604FF0050E05EB0C00BCF10F0FC0E9D1
:108D180001EE00F2328150681546144B1A688A42F7
:108D280038BF1960124B1A688A4238BF196094E03C
:108D3800AA1943F0010346F001066E602046BA60A6
:108D4800536000F043F90835284603B0BDE8F08FBA
:108D5800D9681A44A1E600BF540400245C04002426
:108D68005C08002460440024304400245844002453
:108D78005C440024B2F5206F4FEA522363D3142BCE
:108D880000F2B78003F15C01C9005B3307EB010E09
:108D98007958AEF1080E8E4500F091804B6823F0AB
:108DA8000303934202D989688E45F7D1D1F80CE0C4
:108DB8007A68C5E9021ECEF80850CD60D6E6142BB5
:108DC80059D9542B00F29D80330B03F16F0003F146
:108DD8006E0CC3008AE60EF1010E1EF0030F05F1BA
:108DE80008057FF4D5AE51E0424445465368D8F8AB
:108DF8000C1043F00103536055F8083F2046D96032
:108E08008B6000F0E3F8F3E6F00806F1080237E6B5
:108E18002A442046536843F001035360083500F0A4
:108E2800D5F8E5E6A919204646F0010643F0010405
:108E38006E60C7E90411C1E902CC4C60AB5000F088
:108E4800C5F80835D4E6930903F13901C900383368
:108E58009CE7BD425FD0BD68686820F003084645BE
:108E6800A8EB060302D80F2B3FF762AF204600F0AD
:108E7800ADF80025BCE603F15C0003F15B0CC30010
:108E880034E659F808394B4540F0968010F0030F46
:108E980000F1FF30F5D17B6823EA01037B604900CC
:108EA80099423FF6C0AE19B9BDE649000EF1040E6D
:108EB8001942FAD0704667E603F11008D0E69A1016
:108EC8004FF001087B6808FA02F21A437A6070E7EB
:108ED80002EB08014942C1F30B0A514620460092B1
:108EE80000F07AF8431CDDE900237FF4EFAEDA46A0
:108EF800EFE6542B25D8130B03F16F01C9006E332D
:108F080044E7B3F5AA7F25D8F30B03F1780003F102
:108F1800770CC300EAE5294B186840441860B1E6AD
:108F2800CAF30B0CBCF1000F7FF4ACAEBD68C844AB
:108F380048F001006860F0E61546EEE6012353604C
:108F480094E7B3F5AA7F23D8D30B03F17801C900BE
:108F580077331BE740F25452934223D8B30C03F102
:108F68007D0003F17C0CC300C0E5ABF1080BD844CD
:108F7800A8EB02084FF0000AABE605F1080120460D
:108F88000093FFF703FCBD68009B68681968C4E696
:108F980040F254518B420BD8930C03F17D01C90068
:108FA8007C33F3E64FF47E737F204FF07E0C9DE513
:108FB8004FF47E717E23E9E67B6870E73044002435
:108FC8000148FFF711BD00BF244400240148FFF702
:108FD8000DBD00BF2444002438B5074D00220446C7
:108FE80008462A60F9F71AFB431C00D038BD2B68E5
:108FF800002BFBD0236038BD6444002410B50C4618
:10900800B1F90E1000F040F9002803DB236D03448A
:10901800236510BDA38923F48053A38110BD00BF2D
:109028002DE9F0410C46B1F90C101F46CB05054659
:1090380016460BD421F48051A1813B46B4F90E1099
:1090480032462846BDE8F04100F01EB8B4F90E10CB
:109058000223002200F002F9B4F90C10EAE700BF7D
:1090680010B50C46B1F90E1000F0F8F8A389421CAF
:109078000EBF23F4805343F480532065A38110BDB1
:10908800B1F90E1000F05CB838B50C46084D8446AE
:10909800114620461A4600232B606446F9F79EFCC9
:1090A800431C00D038BD2B68002BFBD0236038BD93
:1090B800644400242DE9F047DFF87CA00646DAF87E
:1090C800000098460F469146FFF78EFC1B4B1B6825
:1090D800D3F8484124B365681F2D26DC5EB96B1CA4
:1090E8000235DAF80000636044F82570FFF77EFC6B
:1090F8000020BDE8F08704EB85010123C1F88890C2
:10910800D4F88821AB401A43022EC4F88821C1F84C
:109118000881E4D1D4F88C211343C4F88C31DEE7FC
:1091280003F5A674C3F84841D5E7DAF80000FFF75D
:109138005DFC4FF0FF30DCE750040024389800084D
:1091480038B5074D0022044608462A60F9F75CFA4C
:10915800431C00D038BD2B68002BFBD0236038BDE2
:109168006444002470B500294BD006460C4610B163
:10917800836B002B48D0636ED80734D5B4F90C3014
:10918800002B3ED021463046FFF744F9E36A0546F6
:1091980033B1E169304698470028B8BF4FF0FF3532
:1091A800A3891A063BD4216B41B104F140039942CB
:1091B80002D03046FFF7EAFA00232363616C21B13D
:1091C8003046FFF7E3FA00236364FFF76DFA636E36
:1091D8000022DB07A28127D5A06DFFF703FCFFF76C
:1091E80069FA284670BDA3899905CBD4A06DFFF70D
:1091F800FBFBB4F90C30002BC4D1656E15F00105EA
:1092080008D00025284670BDFFF7C8F9636ED80757
:10921800B4D4E8E7A06DFFF7E9FB284670BD2169E3
:109228003046FFF7B3FABEE7A06DFFF7DFFBD3E7E1
:1092380070B50C46084D03460026204611461C46CC
:109248002E60F9F7E4F9431C00D070BD2B68002BA1
:10925800FBD0236070BD00BF6444002438B50C46C1
:10926800084D8446114620461A4600232B60644662
:10927800F9F7D2F9431C00D038BD2B68002BFBD07E
:10928800236038BD6444002438B50C46084D844634
:10929800114620461A4600232B606446F9F7A4F9C4
:1092A800431C00D038BD2B68002BFBD0236038BD91
:1092B8006444002438B5C1F30A55A5F2FF32132AD5
:1092C8000B4684468E4604461EDC002A0EDB1D49EA
:1092D800114103EA0100204313D04FF4002343FA5D
:1092E80002F296442EEA010E002408E001F0004E36
:1092F800013204BF4EF07F5E4EF4401E00247346D8
:10930800A4466046194638BD332A08DDB2F5806F99
:10931800F7D10246F6F7E2FF84460B46F1E7A5F2DD
:1093280013454FF0FF3121FA05F52842E9D0012312
:10933800C2F1330203FA02F2841828BF9E4424EAD9
:109348000504DCE7FFFF0F00F8B504460D4600F002
:1093580037F806460F462046294600F035FA78B118
:1093680011A3D3E9002320462946F7F7FDFB50B99E
:109378000FA3D3E9002320462946F7F7D7FB58B9AE
:1093880030463946F8BDFEF7E1FE0B4F2223002692
:10939800036039463046F8BDFEF7D8FE2223036045
:1093A80000260027ECE700BFEF39FAFE422E864080
:1093B80051302DD5104987C00000F07F0000000013
:1093C8002DE9F04FD24F21F00042BA4287B005464E
:1093D8000C464FEAD1760DD9CE4FBA4273D9C1F3B4
:1093E80013030343024640F05781002E66D0002540
:1093F8002C4663E0C84B9A4200F21F81C74B9A4241
:1094080040F235812A46234628462146F7F71CF9BB
:10941800A9A3D3E9002306460F46F7F715F9A8A331
:10942800D3E90023F6F758FF32463B46F7F70CF925
:10943800A5A3D3E90023F6F751FF32463B46F7F7D9
:1094480003F9A3A3D3E90023F6F746FF32463B46C8
:10945800F7F7FAF8A0A3D3E90023F6F73FFF32465F
:109468003B46F7F7F1F802460B4628462146F6F741
:1094780033FFCDE90401DDE9048928462146424647
:109488004B46F7F7E1F8002206460F464FF08043B7
:1094980040464946F6F720FF02460B463046394615
:1094A800F7F7FCF92A462346F6F716FF02460B465D
:1094B80000209B49F6F710FF05460C462846214632
:1094C80007B0BDE8F08F86A3D3E90023F7F74CFB7C
:1094D8000746002840F0EA8083A3D3E90023284602
:1094E8002146F7F723FB002840F037818D4B2846AB
:1094F80003EBC60621467EA3D3E90023F7F7A4F8B9
:10950800D6E90023F6F7EAFEF7F738FB0190F7F7FC
:1095180031F879A3D3E9002306460F46F7F794F804
:1095280002460B4628462146F6F7D6FE74A3D3E931
:1095380000238046894630463946F7F785F8CDE955
:109548000201DDE9022340464946F6F7C5FE024618
:109558000B4682468B4605460C46F7F775F856A328
:10956800D3E9002306460F46F7F76EF854A3D3E96C
:109578000023F6F7B1FE32463B46F7F765F852A3EB
:10958800D3E90023F6F7AAFE32463B46F7F75CF824
:109598004FA3D3E90023F6F79FFE32463B46F7F781
:1095A80053F84DA3D3E90023F6F798FE32463B461D
:1095B800F7F74AF80B46024659465046F6F78CFE2E
:1095C800019B06460F46CDE90467002B3FF453AFD5
:1095D80032463B4650465946F7F736F83246044677
:1095E8000D463B4600204FF08041F6F775FE0246D7
:1095F8000B4620462946F7F751F902460B46DDE9A6
:109608000201F6F769FE42464B46F6F765FE02464A
:109618000B4600204249F6F75FFE019C6FF47F730A
:109628009C420246C0F2868001EB045305461C4664
:109638002846214607B0BDE8F08F3B4B9A423FF6DB
:1096480055AF3A4B03EBC603D3E90023F6F744FEC4
:10965800374BF4002344D3E90034C6F1010ACDE9BD
:109668000234AAEB060380468946019369E726A3DC
:10967800D3E90023F6F732FE294B0022F7F774FAF4
:1096880000283FF4BFAE28462146254B0022F6F7B6
:1096980025FE05460C4611E70B46F6F71FFE054664
:1096A8000C462846214607B0BDE8F08F002007B0D9
:1096B800BDE8F04F00F082B8D0A4BE726937663EAC
:1096C800F16BD2C541BDBB3E2CDE25AF6A56113FBA
:1096D80093BDBE166CC1663F3E5555555555C53FA1
:1096E800EF39FAFE422E864051302DD5104987C0F9
:1096F800FE822B654715F73F0000E0FE422EE63F4D
:10970800763C7935EF39EA3D9C7500883CE4377E34
:10971800412E8640FFFFEF7F422ED63FFFFFEF3DF1
:109728000000F03F40980008B1A2F03F50980008B0
:1097380060980008019800F57A7A01EB0A53104600
:10974800194600224FF0B873F6F77EFF05460C461F
:109758002846214607B0BDE8F08F384607B0BDE877
:10976800F04F00F025B800BFD0B506460F461446A6
:10977800FEF7ECFC0346394630461C60D0BD00BFFE
:1097880030B583B080B1144603F10045CDE90045FA
:1097980010461946DDE90023F6F756FF222203B0EA
:1097A800BDE83040FFF7E0BF14461D46EEE700BFB6
:1097B80000224FF08053FFF7E3BF00BF00224FF0B5
:1097C800E043FFF7DDBF00BF41F0004000F5801027
:1097D800C00F7047F8B500BFF8BC08BC9E4670477C
:0C97E800F8B500BFF8BC08BC9E467047F6
:1097F800000000000102030401020304060708092F
:1098080000061016000610160100020004000600EB
:1098180008000A000C001000200040008000000131
:109828000804020408010101010101030701000005
:109838002800002400000000000000000000E03FB5
:10984800000000000000E0BF0000E0FE422EE63FFE
:109858000000E0FE422EE6BF763C7935EF39EA3D5E
:08986800763C7935EF39EABDC9
:089870007079FF7F0100000088
:08987800FD830008BD02000899
:049880009902000841
:10988400010000000100000014000000A306000015
:109894000090D0030090D0030100000010000000ED
:1098A400280000240000000000000000140300242D
:1098B4007C030024E40300240000000000000000F6
:1098C4000000000000000000000000000000000094
:1098D4000000000000000000000000000000000084
:1098E4000000000000000000000000000000000074
:1098F4000000000000000000000000000000000064
:109904000000000000000000000000000000000053
:109914000000000000000000000000000000000043
:109924000000000000000000000000000000000033
:109934000000000000000000000000000000000023
:109944000000000000000000000000000000000013
:1099540001000000000000000E33CDAB34126DE6B0
:10996400ECDE05000B000000000000000000000019
:1099740000000000000000000000000000000000E3
:1099840000000000000000000000000000000000D3
:1099940000000000000000000000000000000000C3
:1099A40000000000000000000000000000000000B3
:109CD400204400240000000000000000540400247C
:109CE400540400245C0400245C0400246404002460
:109CF400640400246C0400246C0400247404002410
:109D0400740400247C0400247C04002484040024BF
:109D1400840400248C0400248C040024940400246F
:109D2400940400249C0400249C040024A40400241F
:109D3400A4040024AC040024AC040024B4040024CF
:109D4400B4040024BC040024BC040024C40400247F
:109D5400C4040024CC040024CC040024D40400242F
:109D6400D4040024DC040024DC040024E4040024DF
:109D7400E4040024EC040024EC040024F40400248F
:109D8400F4040024FC040024FC040024040500243E
:109D9400040500240C0500240C05002414050024EB
:109DA400140500241C0500241C050024240500249B
:109DB400240500242C0500242C050024340500244B
:109DC400340500243C0500243C05002444050024FB
:109DD400440500244C0500244C05002454050024AB
:109DE400540500245C0500245C050024640500245B
:109DF400640500246C0500246C050024740500240B
:109E0400740500247C0500247C05002484050024BA
:109E1400840500248C0500248C050024940500246A
:109E2400940500249C0500249C050024A40500241A
:109E3400A4050024AC050024AC050024B4050024CA
:109E4400B4050024BC050024BC050024C40500247A
:109E5400C4050024CC050024CC050024D40500242A
:109E6400D4050024DC050024DC050024E4050024DA
:109E7400E4050024EC050024EC050024F40500248A
:109E8400F4050024FC050024FC0500240406002439
:109E9400040600240C0600240C06002414060024E6
:109EA400140600241C0600241C0600242406002496
:109EB400240600242C0600242C0600243406002446
:109EC400340600243C0600243C06002444060024F6
:109ED400440600244C0600244C06002454060024A6
:109EE400540600245C0600245C0600246406002456
:109EF400640600246C0600246C0600247406002406
:109F0400740600247C0600247C06002484060024B5
:109F1400840600248C0600248C0600249406002465
:109F2400940600249C0600249C060024A406002415
:109F3400A4060024AC060024AC060024B4060024C5
:109F4400B4060024BC060024BC060024C406002475
:109F5400C4060024CC060024CC060024D406002425
:109F6400D4060024DC060024DC060024E4060024D5
:109F7400E4060024EC060024EC060024F406002485
:109F8400F4060024FC060024FC0600240407002434
:109F9400040700240C0700240C07002414070024E1
:109FA400140700241C0700241C0700242407002491
:109FB400240700242C0700242C0700243407002441
:109FC400340700243C0700243C07002444070024F1
:109FD400440700244C0700244C07002454070024A1
:109FE400540700245C0700245C0700246407002451
:109FF400640700246C0700246C0700247407002401
:10A00400740700247C0700247C07002484070024B0
:10A01400840700248C0700248C0700249407002460
:10A02400940700249C0700249C070024A407002410
:10A03400A4070024AC070024AC070024B4070024C0
:10A04400B4070024BC070024BC070024C407002470
:10A05400C4070024CC070024CC070024D407002420
:10A06400D4070024DC070024DC070024E4070024D0
:10A07400E4070024EC070024EC070024F407002480
:10A08400F4070024FC070024FC070024040800242F
:10A09400040800240C0800240C08002414080024DC
:10A0A400140800241C0800241C080024240800248C
:10A0B400240800242C0800242C080024340800243C
:10A0C400340800243C0800243C08002444080024EC
:10A0D400440800244C0800244C080024FFFFFFFF20
:04A0E4000000020076
:0400000508002A0DB8
:00000001FF
